:100200004F726967696E616C2046696C653A20704F
:10021000726F6A6563742E6865780D0A4F75747025
:10022000757420446174653A20323030392F30388B
:100230002F31320D0A4F75747075742046696C65E4
:100240003A206B6C38352E6865780000000000009D
:10025000000000000000000000000000000000009E
:10026000000000000000000000000000000000008E
:100270000000000000000000000000000000004539
:10006E000D0A0D0A205B4B4C38355D0D0A0D0A004A
:10007E000D0A0D0A00557365204B4C383543204947
:10008E004F20446566696E650D0A0045444944205B
:10009E004D6978696E6720416C676F726974686D1F
:1000AE00204368616E676520746F204D6F64652014
:1000BE0025640D0A0054524547203D2030782530E6
:1000CE002E32580D0A0043757272656E7420536598
:1000DE006C65637465643A2000527820434B206946
:1000EE006E707574207465726D696E6174696F6E71
:1000FE0020303D35306F686D2C20313D3130306F02
:10010E00686D005278204257207265647563746979
:10011E006F6E00455120626961732063757272655E
:10012E006E7420303D31303075412C20313D3132EE
:10013E00357541005478207072652D656D70686557
:10014E007369732028434C4B2900547820616374E3
:10015E00697665207065616B696E67005478205012
:10016E006C6C204257005478207072652D656D704E
:10017E00686573697320284461746129005478207E
:10018E0035302D6F686D207465726D696E6174699E
:10019E006F6E002842697420256429203D20256455
:1001AE000D0A00416C6C204F757470757420456E8D
:1001BE0061626C650D0A00416C6C204F7574707530
:1001CE007420446973616C650D0A00028000400062
:1001DE001000200001000200040008028000400010
:0B01EE001000200001000200040008C7
:0C91E40041F9A90041F9B40041F9030071
:10996F0075F021A42404F974F935F0FAEBF0A3EAA9
:10997F00F0A3E9F0227AFF798090F901E0FD7B01F5
:10998F0090FC0CE4F0A32290FD98E0FF7401A8076F
:10999F00082290FD97E075F021A42409F582E434A4
:1099AF00F9F583E02275F002A42401F974F935F07A
:1099BF00FA7B012275F021A42404F582E434F9F531
:1099CF0083E02290FD97E0FFC32290FD97E004F023
:1099DF00227BFFE0FF90FAF3E4F0A3EFF02290FD7B
:1099EF0097E075F084A4FFAEF0227B017AF9792518
:0199FF002245
:1053C400E490FD97F0A3F0A374FFF07F0512B5AB52
:1053D400E4F5207DFF7F05127BD67B027DFF7F05F0
:1053E40012694A7D047F06127A6F7B027D077F066D
:1053F40012694AE4FB7D017F0A12694AE4FB7D03DA
:105404007F0C12694AE4FB7D087F0612694AD2AF19
:1054140075FF387BFF7AB4797A12B5B7E4FF12AC22
:105424000A7D017F407E021294917BFF7A00796E9F
:1054340012A8397BFF7A02790012A8397BFF7A001F
:10544400797E12A8397BFF7AB679227F0312B5D907
:105454007B007C077DD01279047BFF7A007983126C
:10546400A83990FD2074FFF0A37401F0A374E9F04F
:105474007B017AF8790012ADEF7D0C7F0B127BD69D
:105484007B017D0C7F0B12694A7D017F08127BD65C
:105494007B027D017F0812694A1298417D017F08D1
:1054A400127A6F7F0112B5AB7B017AF97904E4FDBE
:1054B4001283407B017AF979887DE01283407B0175
:1054C4007AF979677DE51283407B017AF979467D23
:1054D400EA1283401299F97DEF1283407FE01201B2
:1054E400F97B017AF979017D701295D27AF979AA5A
:1054F4007D601257B27AF979AC7DE012A03B7AF95B
:1055040079AE7DE21257B27AF979B07DE412A03B0C
:105514007B017AF979B27DE612A03BE490FD97F025
:105524001299D294015075EF1299B4C003C002C00D
:1055340001E090FC1712996F1299ED2425F974F982
:105544003EFA90FC1A12997B74462FF974F93EFACC
:10555400A312997BD001D002D0031287AE90FD979D
:10556400E01299B4C003C002C001E090FC23129978
:105574006F1299ED2467F974F93EFA90FC2612999A
:105584007B74882FF974F93EFAA312997BD001D069
:1055940002D003128EE91299D902552490FD267483
:1055A40001F0A374F9F0A37404F07B017AF979AAE9
:1055B40012B4C9E490FD97F01299D294045036EFD6
:1055C40075F002A424ACF974F935F0FA7B01C00338
:1055D400C002C001E075F021A42425F974F935F066
:1055E400FA90FD2612997BD001D002D00312B4C9DF
:1055F4001299D980C3E4FFFE12B423EFD39403E4D9
:10560400400690FD60F0800AFFFE12B42390FD6016
:10561400EFF07A00799990FD601299E012A8392090
:1056240008030257ACC20890FD977401F0E4A3F09C
:105634001299D2940540030256DBEF1299C3FB7012
:10564400391299A1FC30E40C1299968002C333D824
:10565400FC0256BAEC30E51790F9A9E075F0148411
:10566400E5F070691299968002C333D8FC80361233
:1056740099968002C333D8FC804DEB6405600B908F
:10568400FD97E01299C3640C70341299A130E61DA1
:1056940090F9A9E075F02884E5F0703112999680AC
:1056A40002C333D8FCFD7F05126C26802012999624
:1056B4008002C333D8FCFD7F05127BD6800F12997C
:1056C400968002C333D8FCFD7F05127A6F1299D9F4
:1056D400A3E004F002563490F9A9E004F0C394C89E
:1056E4004002E4F07B017AF97904123A0590FD97BF
:1056F4007401F01299D294055017EF75F021A42487
:1057040004F974F935F0FA7B011225811299D980D4
:10571400E2E520B40F0B7D047F06127A6F7D0280D0
:10572400097D027F06127A6F7D047F06127BD67B89
:10573400017AF9790112ADBDEF7D017F0660051292
:105744007BD68003127A6F90FD99E025E0F0E0FEAD
:105754007D087F061297A8EF60047F0180027F0016
:10576400EE4FFF90FD99F0BF7F0EE520B40F047F4C
:105774000980027F1212A4A830090AC2097F01120B
:10578400B0C112A4A8124510200D0302562390F9AB
:10579400B4E0FF04F0EFD394325003025623C20D59
:1057A4007F0912A4A80256234387010256237B01D2
:0657B40012A03B7B012264
:1082500090FE0F7406F07AFE790F12998804F0A34D
:10826000F0E4FF12775990F901E004FD7B017AFEFA
:10827000791012998F04F0E4A3F0FF1277597A0075
:1082800079C390FE101299E012A8397BFF7A007929
:10829000D412A83990F903E0B4080050609082A489
:1082A000F82828730282BC0282C40282CC0282D4E3
:1082B0000282DC0282E40282EC0282F47BFF7A001A
:1082C00079E780367BFF7A017911802E7BFF7A0176
:1082D000792180267BFF7A017942801E7BFF7A011B
:1082E000795880167BFF7A01796A800E7BFF7A01CC
:1082F000797480067BFF7A01798B12A8397BFF7A2B
:108300000179A190F903E0FFFC3395E090FAF3F0D6
:10831000A3CCF074017E00A807088005C333CE33D8
:10832000CED8F9FF90FE10E0FDEF5D7E0060047F87
:108330000180027F0090FAF5EEF0A3EFF002A83979
:10A4A800EF24EE602B2409704E7BFF7A0179B112FC
:10A4B800A839E4F5201299F912B5CE7AF97946123D
:10A4C800B5CE7AF9796712B5CE7AF9798802B5CE20
:10A4D8007BFF7A0179C512A83975200F1299F912F4
:10A4E800B5C37AF9794612B5C37AF9796712B5C353
:08A4F8007AF9798812B5C3223C
:10A3900090FE11EFF0A3EDF090FF807406F012999B
:10A3A0008404F0A3F0E4FF12775990F901E004FD72
:10A3B0007B017AFF798112998F04F0E4A3F0FF12F8
:10A3C000775990FE12E090FF81600BE0FF90FE1144
:10A3D000E0FEEF4E800AE0FF90FE11E0F4FEEF5E3B
:10A3E00090FF81F01299847402F0E4A3F0FF0277E9
:01A3F0005913
:10B47A00AE07E4FF12B0C1BF8609EE7006EDB41044
:04B48A0002D20922BF
:03B62200D2082229
:103FB90000000000000000000000000000000000F8
:103FC9000000D60980A020E02D101060A200040393
:103FD900000000188C0AD08A20E02D10103E9600AF
:103FE9000403000000188C0AD08A20E02D10103E2E
:103FF9009600100900000018011D007251D01E2002
:104009006E28550010090000001E011D8018711C42
:104019001620582C250010090000009E8C0AA014B7
:1040290051F01600267C43000403000000988C0A16
:10403900A01451F01600267C4300100900000098D6
:104049008C0AA01451F01600267C430004030000DA
:1040590000188C0AA01451F01600267C43001009A0
:104069000000001818154028B2F016004CF843005B
:1040790004030000009818154028B2F016004CF807
:10408900430010090000009818154028B2F01600E6
:104099004CF8430004030000001818154028B2F03A
:1040A90016004CF843001009000000181815A01458
:1040B90051E02D10207C960004030000001818150B
:1040C900A01451E02D10207C960010090000001862
:1040D900023A801871382D40582C4500100900000B
:1040E900001E8C0AD090204031200C40550004035A
:1040F900000000188C0AD090204031200C40550057
:10410900100900000018011D00BC52D01E20B8285B
:10411900554010090000001E011D80D0721C162098
:10412900102C258010090000009E8C0AA020512027
:104139001810187E23000403000000988C0AA020A0
:1041490051201810187E23001009000000988C0ACD
:10415900A02051201810187E230004030000001825
:104169008C0AA02051201810187E23001009000085
:10417900001818154040B220181030FC2300040321
:104189000000009818154040B220181030FC230098
:1041990010090000009818154040B220181030FC92
:1041A900230004030000001818154040B22018101D
:1041B90030FC23001009000000181815A0205140F8
:1041C90031201880550004030000001E1815A02096
:1041D900514031201880550010090000001E023A94
:1041E90080D072382D40102C458010090000001E27
:1041F900011D803E73382D407E2C4580100900003A
:10420900001E011D80D072382D40102C45801009E8
:104219000000001E011D80D072382D40102C4580F1
:1042290010090000001E3B2A4028B2E02D1060F85A
:1042390096000403000000183B2A4028B2E02D1024
:1042490060F89600100900000018302A4040B2407A
:10425900312030005510040300000018302A404076
:10426900B240312030005510100900000018201C00
:104279008080711C552020A8750410090000009A3F
:10428900023A80D0721C1620102C258010090000DB
:10429900009E023A00BC52D01E20B8285540100991
:1042A9000000001E1815D090204031200C40550008
:1042B9000403000000181815D090204031200C404C
:1042C90055001009000000181815D090202018106A
:1042D900187E23000403000000981815D0902020B0
:1042E9001810187E2300100900000098023A80185F
:1042F900711C1620582C250010090000009E023A56
:10430900007251D01E206E28550010090000001EB1
:104319001D15D08A20E02D10103E960004030000E0
:1043290000181D15D08A20E02D10103E96001009A6
:10433900000000181D15A01451F01600267C43003A
:104349000403000000981D15A01451F01600267CE6
:104359004300100900000098302AD09020403120F5
:104369000C405500040300000018302AD09020406A
:1043790031200C405500100900000018302AA020F7
:1043890051201810187E2300040300000098302AD9
:10439900A02051201810187E230010090000009851
:1043A9003B2AD08A20E02D10103E9600040300001D
:1043B90000183B2AD08A20E02D10103E96001009E3
:1043C900000000183B2AA01451F01600267C430077
:1043D9000403000000983B2AA01451F01600267C23
:1043E900430010090000009800FFFFFFFFFFFF00D6
:1043F9001710010901000000000E010380734178C4
:104409002A7C119E59479B2710505421080001010D
:104419000101010101010101010101010101011D67
:10442900007251D01E206E28550010090000001E90
:104439008C0AD08A20E02D10103E9600040300005B
:104449000018000000FC0045502D48444D492D52EC
:10445900580A2020000000FD003B3D0F2E08000AED
:1044690020202020202001AB02031D714A8405135E
:1044790014010203111210230907078301000065C3
:10448900030C001000023A801871382D40582C4551
:104499000010090000001E011D8018711C1620580B
:1044A9002C250010090000009E011D00BC52D01EE1
:1044B90020B828554010090000001E011D80D07247
:1044C9001C1620102C258010090000009E8C0AD093
:1044D90090204031200C40550004030000001800D2
:1044E900000000000000001E8102031112040907E8
:1044F90007010000030C001000881E097F07170739
:07450900503F06C04F000007
:0491F00041FD6000DD
:1057BA005FFFE0FBA3E0FAA3E0F9900001EF121B00
:1057CA00B990FBCAE02402FFE433FE90FBC1E0FB80
:1057DA00A3E0FAA3E0F98F828E83121B58FF90FB95
:1057EA00C9E02402FDE433FC90FBC4E0FBA3E0FA29
:1057FA00A3E0F9228D828C83121B58FF90FBC1E033
:10580A00FBA3E0FAA3E02480F9E43AFA90FBCAE0A9
:10581A002290FBCAE0FFF582758300021B58E42937
:10582A00F9EA3401FA121B3F54FE121BA790FBC17E
:10583A00E0FBA3E0FAA3E0228F828E83121B58FFBB
:10584A00227F807E00121B1990FBC87401F022FE91
:10585A0004F0EE7C0029F9EC3AFAEF021BA78D82DC
:10586A008C83021B5890FBCEE0FE04F08E82758377
:10587A0000EF021BB990FBC9E0FF90FD62E02FFF29
:10588A0090FD61E034002290FBCEE0FF90FD61E0E4
:10589A00FCA3E0FDC39F7480F8EC6480982290FC1E
:1058AA00457401F0A374FBF0A374CFF090FBD8E029
:1058BA00F9A3E0FAA3E090FC48C9F0A3EAF0A3E94F
:1058CA00F02290FBCC541FFEEF2EF02290FBC9E091
:1058DA00FF7E0090FD61E0FCA3E0FD2FFFEE3CFEA1
:1058EA0022FF90FD5FE02FF090FD62E004F02212AB
:1058FA001BB9E490FD5FF090FD61F0A3F022541F04
:10590A00FEEF2E90FBCBF090FBC9E004F022900052
:10591A0083121B5854C0440190FBCDF090FCD874FC
:10592A0001F0A374FBF0A374CEF090FBD22290FD99
:10593A0061E0FEA3E0FF2290FBCCE0FF90FBCAE00F
:10594A00FED39F2290FD61E004F022E0FFC390FDA8
:10595A0062E09F7480F890FD61E06480982290FB79
:10596A00CAE004F022E429F9EA3401FA121B3F548E
:10597A00FD021BA790FBCAE0FF04F08F8222FF04FE
:10598A00F07E00E92FF9EE3AFA2290007E121B58B7
:10599A00640122900001EF121BB990FBC122F8ACFE
:1059AA0002AD037BFF228D828C83EF021BB990FB31
:1059BA00CA7484F022EF900002021BB9900001120F
:1059CA001B58FF90FBC12290FBCBE0FF90FBC9E084
:1059DA002290FBC9E02402FFE433FE2290FBCFE0D1
:1059EA002402FDE433FC90FBD522121BA790FBCACC
:1059FA00E02401FFE433FE2290FD61E0FCA3E022F3
:105A0A00EF2402FFE43EFE222480F9E43AA801FCD6
:105A1A00AD032290FBC97484F02290FD5FE014F478
:105A2A00FF90FBC1222FF582E43EF583021B581238
:105A3A001B3FFF90FBC9E024012290FBCAE0FD90C6
:105A4A00FD62E02DFD22900100021B5890FD60E0EE
:105A5A00640322900023021B58EF121BA790FBC17C
:105A6A0022900024021B58900025021B5890000126
:105A7A00121B586D22900002121B586F227E00FDE5
:105A8A00EE33FC90FBC122C390FBD0E0940522C305
:105A9A00947FEE6480948022900082021B58A3F0C7
:105AAA00A3EBF0A3222480F9E43AFA22900036020A
:105ABA001B58900037021B58FC8D82F583021B5835
:105ACA0090FBCEE0C3941E2290FBCFE0C3942D221C
:105ADA0090FBC9E02403F02290FBCCE0FF90FBCAC4
:105AEA00E0D39F228F828E83021B5890FBD0E0C3A3
:105AFA00940C227405121BA790FBDE222400F9EAFB
:105B0A003401FA021B3F2DF582E43CF583021B584F
:105B1A00E0FBD3EF9B7480F86E9822541FFF90FD30
:105B2A0062E02FF02290007E021B589FEE6480F8FC
:105B3A00EC64809822121BA790FBDB2212245B7E66
:105B4A00007F037D0022E0FFFDC390FD62E09D22FD
:105B5A00541FFEEF2E90FBCBF02290FBCFE0F58294
:105B6A0075830022121BA790FBD82290FBC9E0FD87
:055B7A007C00EF2D226C
:10A44F0090FD9AEB1258C490FD9A1257F5EA494BBA
:10A45F00604690FD9A12583A1259A87A4379F17EC4
:10A46F00017F00121B1990FBC474FFF0A37443F01B
:10A47F00A374F1F0E4A3F090FD9A1257F512028045
:10A48F0090FD9A12583A125B064401121BA7440220
:09A49F00121BA754FB121BA7229B
:109A910090FD9DEB1258C490FD9D1257F5125994FB
:109AA100707990FD61F0A37404F090FD9D1257F55B
:109AB100125AA212589550527480125B1054E064ED
:109AC10060701F7481125B10640370331259382463
:109AD10082125A30640C70277483125A2F70207FBF
:109AE100012290FD9D1257F590FD62E024801258ED
:109AF100898F82F583121B58125B2512588AF01246
:109B010058F270A612594E029AAB90FD9D1257F56C
:0E9B1100125AA212595640037F00227F0022F2
:109F490090FD44EDF090FD41EB1258C4125B2FC314
:109F59009401406290FD45E0FF90FD61E4F0A3EFBC
:109F6900F090FD411257F5125AA22480FFE433FE06
:109F7900125A02FDC3125B355023125868FE54E091
:109F8900FF90FD44E0B50703AF0522EE125B2512F1
:109F9900588AF01258F270C912594E80C490FD4186
:109FA9001257F5125AA22480FFE433FEC3ED125B67
:099FB9003540037F00227F0022E5
:10B10F0090FCD5EB1258C490FCD512583A1259A89E
:10B11F007A4479F17E007F06121B1990FCD81257E2
:06B12F00F57406021BA7E7
:10AB5C0090FC42EB1258C490FC4212583A1259A87D
:10AB6C007A4479F77E007F03121B1990FC4512572B
:10AB7C00F57403121BA790FC4812583A1259A87A84
:0AAB8C004479FA7E007F03021B19D2
:10B1350090FCDBEB1258C490FCDB12583A1259A86C
:10B145007A4479FD7E007F07121B1990FCDE1257A9
:06B15500F57407021BA7C0
:10AB960090FC4BEB1258C490FC4B12583A1259A831
:10ABA6007A4579047E007F09121B1990FC4E1257D4
:10ABB600F57409121BA790FC5112583A1259A87A3B
:0AABC60045790D7E007F03021B1984
:1002800090FBC1EB1258C4E490FBC8F07B0190FBDB
:10029000D204F0A374FFF07480125AA874FFF074B3
:1002A0009E125AA874FFF0A374CBF0A3EBF0A374D2
:1002B000FFF0A374CEF0A3EBF0A374FFF0A374DA05
:1002C000F090FBC11257F5EA494B7002FF2290FDF6
:1002D00060E0640260030203A690FBC11257F512AE
:1002E0005A5020E0030218F3125828F8AC02AD036C
:1002F000A31257F512584B1257F212599460030289
:1003000018F390FBC11257F5125A5020E10302185E
:10031000F312596F90FBC412583A125AAFC003C07F
:1003200002C001125837125A12D001D002D0031263
:10033000584B90FBC7E030E0030218F390FBC1126A
:1003400057F512196470030218F390FBC11257F5A8
:1003500090FBCAE0125820541FC3940750030218A0
:10036000F3125968E0FF2405125A87A3A3E02DF980
:10037000EA3CFA121B3F548F125B3F1257F5900074
:1003800006121B58FDC3941E500280027D1EEF24EE
:1003900006FFE43EFE90FBC11257F58F828E83ED7F
:1003A000121BB90218F31257F2125B2FD3940140BB
:1003B000037F002290005A121B58707490005B1249
:1003C0001B58706C90005C121B58706490005D129A
:1003D0001B5864FD705A125901125938C39412EE19
:1003E00064809480504A1257F2EF245AFFE43EFE94
:1003F0008F82F583121B5890FBCDF090FD62E024B4
:100400006CFD12588A125AC38F828E83121BB990C8
:10041000FBCDE0FF90FD62E0246CFD12588A8D82D6
:10042000F583EF121BB91258F270AE12594E80A923
:1004300090FBC11257F5125A5030E00F125828F8AD
:10044000AC02AD03A31257F512584B125A56600373
:1004500002051E90FBC11257F5125A5DFF1257F2AA
:10046000125A5D4F4421FF90FBD21257F5125A6386
:100470001257F5125A6BFF1257F2125A6B4F44087B
:10048000FF90FBD21257F512599D1257F5125A716F
:10049000FF1257F2125A714FFF90FBD21257F5120A
:1004A00059BF1257F290006C121B5860030205E20C
:1004B00090006D121B5860030205E290006E121B43
:1004C0005860030205E290006F121B5864FD600340
:1004D0000205E290FBC11257F590006C121B5860A8
:1004E000030205BD90006D121B5860030205BD900C
:1004F000006E121B58702490006F121B5864FD7020
:100500001A900075121B58FF1257F2900075121BBB
:1005100058D39F50030205E20205BA0205BD90FBC5
:10052000C11257F5125A5DFF1257F2125A5D5F441D
:1005300021FF90FBD21257F5125A631257F5125A47
:100540006BFF1257F2125A6B5F4408FF90FBD212F6
:1005500057F512599D1257F5125A71FF1257F212A0
:100560005A715FFF90FBD21257F51259BF1257F222
:10057000125AB6606D125ABCFF606790FBC11257E9
:10058000F5125AB66037125ABCFE6031EFC39E5066
:1005900002802A90FBC11257F5125ABCFF1257F283
:1005A000125ABC6F703C90FBC11257F5125AB6FF3D
:1005B0001257F2125AB6C39F5028E9800690FBC426
:1005C00012583A2436F9E43AFAC003C002C00112C4
:1005D00058372436125A14D001D002D0037F481263
:1005E000584D90FBC11257F5125A5DFF90FBD21285
:1005F00057F5121B3FFE6F70211259C61257F512A4
:100600005A6BB5071590FBD21257F590000212599C
:10061000C91257F5125A716F600312585290FBC1FC
:100620001257F5900023EE121BB990FBD21257F52A
:100630001259C61257F5900024EF121BB990FBD245
:100640001257F59000021259C91257F5900025EF84
:100650001258F9125938125A99501390FBC1125777
:10066000F51258421258EC70EA12594E80E5125AAF
:10067000241257F590007FEF121BB97E007F1E7D7C
:100680000090FBD21257F512245B7E007F2D7D0077
:1006900090FBD51257F5125B4690FBD81257F51216
:1006A000245B7E007F0C7D0090FBDB1257F5125B14
:1006B0004690FBDE1257F512245BE490FBCDF090E0
:1006C000FBCFF090FBCEF090FBD0F0A3F090FBC1FD
:1006D0001257F5125994600302084F1257F2125B39
:1006E0002F600302084F90FBC11257F5125A503089
:1006F000E20302195E900083121B58FF54C04401AC
:1007000090FBCDF06F6003125852125A567040128F
:1007100059B890FBC11257F5121975605090FBC182
:100720001257F512581B1258CC801F12594150E233
:10073000125ACA501590FBC11257F58E82125822D8
:10074000FF90FBD21257F512586F12596880DC9057
:10075000FBC11257F5900084121B58541F640660A9
:10076000031258521259261257F512B10F1259B8E6
:1007700090FBC11257F5121988603590FBC11257D2
:10078000F512581B1258CC802212594150E2125ACD
:10079000D2501890FBC11257F58E82125822FF904A
:1007A000FBD51257F590FBCF12587212596880D9B9
:1007B00090FBC11257F512199B604590FBC112576F
:1007C000F512581B1258CC1259681259811258222E
:1007D000FF90FBD81257F5125A631257F512597E43
:1007E000125822FF90FBD81257F512599D1257F557
:1007F00012597E125822FF90FBD81257F51259BF9A
:1008000090FBC11257F5121964603590FBC1125765
:10081000F512581B1258CC80221259415022125AFC
:1008200091501890FBC11257F58E82125822FF90FA
:10083000FBDB1257F590FBD012587212596880D921
:1008400012585290FD60E060030215B40215A9121F
:1008500057F2125994600302156C1258FD12593860
:10086000C39480EE6480948050121257F274801208
:100870005A2F1258EB70E612594E80E190FD5FE05E
:100880006043125837240012597190FBC11257F57A
:1008900090007E7401121BB91258521257F212596D
:1008A000181257F512B10F1258A890FBD51257F530
:1008B0001219F81257F512B13590FD60E06003028D
:1008C00015B40215A990FBC11257F5125A50FE300B
:1008D000E20302195EEE30E12112596F90FBC4125F
:1008E000583A125AAFC003C002C001125837125A08
:1008F00012D001D002D00312584B1257F29000834D
:100900001259C91257F5900083121B58FE5F54F01C
:10091000444190FBCDF06E6003125852125A56605B
:10092000030209E61259B890FBC11257F512197566
:10093000603290FBC11257F512581B1258CC801F21
:1009400012594150E2125ACA501590FBC11257F584
:100950008E82125822FF90FBD21257F512586F1256
:10096000596880DC125A1D1257F21219AC7003023A
:100970000A9F1257F290FBC912581E90FBCB1258D7
:10098000CF1259111259D1D39F50DCE412590112E0
:10099000589150251257F290FBC9E0125820547F0D
:1009A000FF90FBD21257F5125868547F6F600A12FD
:1009B00058F270DB12594E80D690FBCE125B50126B
:1009C000595D401CEF941E50171257F290FBC9E07E
:1009D000125820FF90FBD21257F512586F1258523E
:1009E000125ADA0209841259B890FBC11257F590D5
:1009F000FBCAE090FD45F07D40121A407003020AE8
:100A00009F90FBC11257F512581B1258CC020A993D
:100A1000125AE250D4125A1D1257F21219AC6079D0
:100A20001257F290FBC912581E125B5A80381259A5
:100A3000D1FED39F503590FBC11257F590FBCAE011
:100A4000125820FF547FFD1257F28E82125822FE58
:100A5000547FB50511125ACA500CEE4FFF90FBD2CD
:100A60001257F512586F12591180C390FBCEE060F7
:100A70002224FFFFE434FFFE90FBD21257F51258F8
:100A80004290FBC11257F590FBCAE01258206F60EC
:100A9000878000125852020A18125968020A1090F0
:100AA000FD60E0FF64016008EF64036003020DADC8
:100AB0001259B890FBC11257F5121988603590FB96
:100AC000C11257F512581B1258CC802212594150AE
:100AD000E2125AD2501890FBC11257F58E8212586A
:100AE00022FF90FBD51257F590FBCF125872125986
:100AF0006880D9125A1D1257F21219BF7003020CE6
:100B00009E1257F290FBC912581E1259081259D161
:100B1000D39F50E2E412590190FBCF125955400384
:100B2000020C3F1257F290FBC9E0125820FF547894
:100B3000FE90FD5FBE0805747FF080037478F0902E
:100B4000FD5FE05FFF90FBD51257F5125A02F58268
:100B50008C83121B58FE90FD5FE05E6F6003020CF9
:100B6000311257F290FBC9E01258205407FFEE549F
:100B700007FED39F4004AF0680001257F290FBC9D6
:100B8000E012582054784FFF90FBD51257F5125AB7
:100B900002FDF5828C83EF121BB990FBC91259FA42
:100BA0001257F212584290FBD51257F5ED2401FD71
:100BB000E43C125AC24F8D828C83121BB9125938F1
:100BC000F5828E83121B585478FDBD082B90FBD5FF
:100BD0001257F5125A0AE92FF9EA3EFAC003C00289
:100BE000C001121B3F1257E71258684FD001D002C4
:100BF000D003121BA7020C3F1259DB1257F21258F6
:100C00004290FBD51257F590FD62E02402FD125888
:100C10008A125AC2FED39F4004AF0680091259DBE4
:100C20001257F212584290FBD51257F51259B08064
:100C30000E90FD62E02403F012588AF0020B189027
:100C4000FBCF125B5012595D404EEF942D5049126C
:100C500057F290FBC912581EFE90FBD51257F512A1
:100C60005B64EE121BB9EF1259FB1257F212584295
:100C7000ED24011259EC1257F51259B01259DB123A
:100C800057F21258421259E61257F51259B090FB1A
:100C9000CFE02403F0125852125ADA020B0D90FBE7
:100CA000C11257F512199B603FE004F090FBC1128E
:100CB00057F512597E125822FF90FBD81257F512A1
:100CC0005A631257F512597E125822FF90FBD81220
:100CD00057F512599D1257F512597E125822FF905E
:100CE000FBD81257F51259BF1257F2121A1E700391
:100CF000020FFCE004F01257F290FBC912581EFEDE
:100D000090FBD81257F5121B3F6E60031258527EAB
:100D100000EF2401FDEE1257F0125868FD90FBD849
:100D20001257F5125A776003125852125A0A125784
:100D3000F212584290FBD81257F5125A7F600312F4
:100D4000585290FBD81257F5C003C002C001121BC5
:100D50003FFF1257F290FBC9E01258204FD001D04C
:100D600002D003125B6E12583A2401F9E43AFAC039
:100D700003C002C001125A391257EE1258684FD000
:100D800001D002D003125B6E12583A2402F9E43A01
:100D9000FAC003C002C001121B3F1257E712586885
:100DA0004FD001D002D003121BA7020FFC1259B87A
:100DB00090FBC11257F590FBCAE090FD45F07D20F5
:100DC000121A407003020F3590FBC11257F51258EA
:100DD0001B1258CC125968125AE250D4125A1D12E2
:100DE00057F21219BF7003020F2B1257F290FBC972
:100DF00012581E1259081259D1FED39F50E11257B2
:100E0000F28E82125822FF5478FE90FD5FBE0805D4
:100E1000747FF080037478F090FBC11257F590FB5B
:100E2000CAE0125820FE90FD5FE0FD5EFCED5F6CB5
:100E30006003020EF4125AD24003020EF4EE54077D
:100E4000FF1257F290FBC9E01258205407FEC39FCF
:100E50005004AF06801090FBC11257F590FBCAE01A
:100E60001258205407FF1257F290FBC9E0FE1258A7
:100E70002054784FFF90FBD51257F5125B64EF12A8
:100E80001BB990FBCAE02401FDE433FC90FBC112C6
:100E900057F5125868FFEE24011257EE1258685F9A
:100EA000FF90FBCFE0FE24011259EC1257F51259C6
:100EB000B08E8212582254786408700A1257CB12EE
:100EC00058685FFF801E1257CB125868FEC39F50B0
:100ED00004AF06800F90FBCA1259DE90FBC1125777
:100EE000F51258421259E61257F51259B090FBCF3D
:100EF000E02403F090FBCFE0FF602724FDFFE43403
:100F0000FFFE90FBD51257F5125AEE547FFF90FB6F
:100F1000C11257F590FBCAE0125820547F6F60054C
:100F20008000125852125ADA020DF690FBCAE024E1
:100F300003F0020DD790FBC11257F590FD45748464
:100F4000F07D80129F4990FBCAEFF07003020FFC06
:100F50001257F2121A1E7003020FFCE004F0A3E015
:100F600004F090FBC11257F590FBCAE0125820FF25
:100F70001257F290FBC9E01258205FFF90FBD81285
:100F800057F5EF1259F490FBC11257F5125842125F
:100F90005A3D1257EE12586890FBD81257BA1258A1
:100FA000685FFF90FBD81257F59000021259A0120B
:100FB00057F512581BFE90FBD81257F5121B3F6EC7
:100FC00060031258527E00EF2401125A891257F51D
:100FD000125868FD90FBD81257F5125A7760031229
:100FE0005852125A0A90FBC11257F512584290FB00
:100FF000D81257F5125A7F6003125852125A56608F
:10100000030211D190FBC11257F5121A0D603590F1
:10101000FBC11257F512581B1258CC8022125941AD
:101020005022125AF5501890FBC11257F58E8212B9
:101030005822FF90FBDB1257F590FBD0125872122A
:10104000596880D91257F2121A2F700302133B12FB
:1010500057F290FBC912581E125908E41259011296
:1010600058D690FBCB125B1A400302133B90FBD087
:10107000E0FFC3ED9FEC64809840030211A8125971
:101080003864064E6018EF64084E6012EF64094E33
:10109000600CEF640A4E6006EF640B4E70771258D6
:1010A000D61257F212584290FBDB1257F5125868CD
:1010B000FED39F4004AF06800A12587FFE1257F2FB
:1010C00012584290FBDB1257F5125A02FDF5828C42
:1010D00083121B586F600312585290FBC9E07E00C8
:1010E0002DFFEE3CFE1257F212584290FBDB1257D6
:1010F000F5125868FED39F4004AF06800A12587F4D
:10110000FE1257F212584290FBDB1257F5125A02A8
:10111000F582021159125938C39405EE6480948007
:10112000503D90FBC7E020E1030211C6125B75FD44
:10113000EC3E1257F1125868FD90FBDB1257F51286
:101140005AEE6D60031258521258D61257F21258C6
:101150004290FBDB1257F58D821259B20211C61272
:1011600058D61257F212584290FBDB1257F512581C
:10117000686F600312585290FD61E0FEA3E029F908
:10118000EA3EFAC003C002C001121B3FFF90FBC938
:10119000125A4712588A1257F11258684FD001D08C
:1011A00002D003121BA7801E125AF5501912587F45
:1011B000FE1257F212584290FBDB1257F590FBD00B
:1011C0001258721258521258F2700312594E0210ED
:1011D0005F90FBC11257F5121A0D700302133B12F8
:1011E00057F2121A2F700302133B1257F290FBC9E9
:1011F00012581E125B5A90FBC11257F512581B125F
:1012000058CC125911A3E004F0E412590190FBCA22
:101210001258D990FBCC125B1A400302131A90FBB0
:10122000C9E0F9FF7E00ED2FFFEE3CFE90FBCBE026
:10123000FDD3EF9D74806E98400302131A125AF585
:10124000400302130F12593864064E6018EF640809
:101250004E6012EF64094E600CEF640A4E6006EFB8
:10126000640B4E7032E9125883FE1257F212584244
:10127000125A4412588AFC90FBC11257F512586852
:10128000FEC39F5005AF060212E512587FFE1257AB
:10129000F21258420212E5125938C39405EE6480E6
:1012A0009480502590FBC7E030E10C125B75FFEC99
:1012B0003EFE90FBC4800A90FBCA125882FE90FB4F
:1012C000C11257F5125842801C12587FFE1257F275
:1012D000125842125A4412588AFC90FBC11257F518
:1012E0001258685FFF90FBDB1257F590FBD0125845
:1012F0007290FBCA1258D990FBC11257F51258428E
:1013000090FBDB1257F51258686F600312585212A7
:1013100058F2700312594E02120D90FBCAE024FFDE
:10132000FFE434FFFE90FBC11257F5125AEE541F32
:10133000FF90FBD0E06F600312585290FBDB125716
:10134000F57403125B3F1257F5900001740C121BE9
:10135000B9E41259C090FBC7E030E21590FBDB12F4
:1013600057F59000037410121BB9900004E4121B8F
:10137000B9125A9150037405F090FBD0E0C3940762
:10138000402E90FBDB12583A2405F9E43AFA121B7E
:101390003F54BF125B3F1257F5900006121B58FFD7
:1013A000C3942D500280027F2D900006EF121BB9CE
:1013B000125A5660030214A91259B890FBC1125771
:1013C000F51219D2604190FBC11257F512581B1249
:1013D00058CC125968E0125820B405DF1259415018
:1013E000DA90FBD1E0C39403501890FBC11257F57B
:1013F0008E82125822FF90FBDE1257F590FBD1121D
:10140000587212596880D5125A1D1257F21219E5F6
:1014100070030215B41257F290FBC912581E1259EC
:101420000812581EB405E37E00EF2401FDEE33FCE4
:10143000125868FD90FBDE1257F5125A77600312BE
:101440005852125A0A1257F212584290FBDE1257A3
:10145000F5125A7F6003125852125AFD12583A245C
:1014600001F9E43AFAC003C002C001125A39125716
:10147000EE1258684FD001D002D003125AFF125812
:101480003A2402F9E43AFAC003C002C001121B3F39
:101490001257E71258684FD001D002D003121BA791
:1014A00090FBD17403F002140A1259B890FBC112D8
:1014B00057F51219D270030215B490FBC11257F5FB
:1014C00012581B1258CC125968E01258206405605B
:1014D000030215B4125A1D1257F21219E5700302D5
:1014E00015B41257F290FBC912581E125908E01297
:1014F0005820640560030215B490FBDE1257F574A2
:10150000051259F490FBC11257F5125842125A3D78
:101510001257EE12586890FBDE1257BA1258685FE5
:10152000FF90FBDE1257F51259BF90FBD17403F008
:1015300090FBCAE0FF2401125A871257F51258682F
:10154000FD90FBDE1257F5125A77600312585212C3
:101550005A0A90FBC11257F512584290FBDE1257FF
:10156000F5125A7F604E1258520215B412583724A1
:101570000012597190FBC11257F590007E74011250
:101580001BB91258521257F21259181257F512B1CC
:101590000F1258A890FBD51257F51219F81257F5EB
:1015A00012B13590FD60E0700B125837125B0644A3
:1015B00004121BA790FBC11257F512599460030245
:1015C00018F390FBCEE0C39401500912592612572C
:1015D000F512B10F90FD60E0B4042990FC4E740147
:1015E000F0A374FBF0A374CFF090FBD8E0F9A3E074
:1015F000FAA3E090FC511258C390FBD51257F51294
:10160000AB96801590FBCFE0C39403500C1258A802
:1016100090FBD51257F512AB5C125A91501790FC03
:10162000DE7401F0A374FBF0A374D0F090FBDB1226
:1016300057F512B13590FBC7E020E009D3125A925A
:1016400040037405F0E4125901125891501690FBB2
:10165000D21257F512586820E70A1258F270EA12AF
:10166000594E80E590FBCE125955400E90FBD21298
:1016700057F5121B3F4480121BA7E490FBCAF012DF
:1016800058061259887402121BA7125806FF04F05C
:1016900012598D7403121BA790FBCFE0FF90FBCE75
:1016A000E02FFF90FBD0E02FFFA3E060047E0F80CF
:1016B000027E0BEF2EFF1258067C0029F9EC3AFA55
:1016C000EF121BA790FBCFE01475F01E84121B8550
:1016D00012596890FBCDE0125805FE04F0EE125846
:1016E0005F90FBCEE04440125805FE04F0EE125825
:1016F0005FE4125901125891501690FBD21257F51F
:101700001257FE1258591258F270EA12594E80E5DB
:1017100090FBCFE0D3941E406F1258061259887484
:101720003E121BA7E4125901125938C3941EEE64ED
:10173000809480501A90FBD51257F58F828E8312B9
:1017400058021258591258F270DE12594E80D99030
:10175000FBCFE024E2FFE434FFFE90FBD512583AC1
:10176000241EF9E43AFAC003C00290FBD5A3E0FAC4
:10177000A3E0F8AC02AD03D002D003121B1990FB1A
:10178000CFE024E2F002171090FBCFE04420125883
:1017900005125859E412590190FBCF125894501673
:1017A00090FBD51257F51257FE1258591258F27085
:1017B000E712594E80E21258061259887483125B60
:1017C0006E1257F5121B3F12580512585990FBD84C
:1017D0001257F5900001125802FE04F0EE12585F05
:1017E00090FBD81257F5900002125802FE04F0EE5A
:1017F00012585F90FBD0E04460125805FE04F0EEF2
:1018000012585FE412590190FBD012589450169070
:10181000FBDB1257F51257FE1258591258F270E7B7
:1018200012594E80E290FBD1E0FFD394004035EF97
:1018300044E0125805125859125806125988125A83
:10184000FD1257F5900001125802FE04F0EE1258F6
:101850005F90FBDE1257F5900002125802FE04F072
:10186000EE12585FE4125901125891505C90FBCA75
:10187000E0C3946E505390FBD21257F5125868543F
:101880007FFF64016038EFC3943C5032EF75F01273
:10189000A424B9F9743F35F0FA7BFFC003C002C03D
:1018A000011258067E0029F9EE125A16D001D00214
:1018B000D0037F12121B1990FBCAE02412F01258B9
:1018C000F2700312594E02186890FBCAE0FFFDC384
:1018D00074809DFDE49400FCC004C00512583712CA
:1018E0005AAFEF7C0029F9EC3AFA7D00D007D00618
:1018F00012245B1258FC125938125A99501390FB5B
:10190000C11257F51258421258EC70EA12594E8023
:10191000E5125A241257F590007FEF121BB91259A5
:1019200094703B90FBC11257F59000FEE41258F9F9
:10193000125938125A995019125837125AAFE92FC2
:10194000F9EA3EFA121B3F1258EB70E412594E802E
:10195000DF125A241257F59000FFEF121BB990FBCB
:10196000C8E0FF2290FD457484F07D60129F49908D
:10197000FBCAEFF02290FBCAE090FD45F07D4012DB
:101980009F4990FBCAEFF02290FBCAE090FD45F022
:101990007D20129F4990FBCAEFF02290FD45748490
:1019A000F07D80129F4990FBCAEFF02290FBC9E0C6
:1019B00090FD45F07D40129F4990FBC9EFF02290C9
:1019C000FBC9E090FD45F07D20129F4990FBC9EFD7
:1019D000F02290FBCAE090FD45F07DE0129F499017
:1019E000FBCAEFF02290FBC9E090FD45F07DE012CC
:1019F0009F4990FBC9EFF02212AB5C90FCDE7401B2
:101A0000F0A374FBF0A374D0F090FBDB2290FD45B3
:101A10007484F07D60129F4990FBCAEFF02290FD24
:101A2000457484F07D80129F4990FBC9EFF02290AD
:101A3000FD457484F07D60129F4990FBC9EFF02250
:091A4000129F4990FBCAEFF0224D
:1030710049646C65005472616E736D69745F4D656E
:103081007373616765005365745F4C6F6769636152
:103091006C5F4164647265737300436F6E6E656348
:1030A1007400446973636F6E6E6563740053746179
:1030B1006E646279005374616E6462795F416C6C15
:1030C100005265636F72645F43757272656E74005E
:1030D1005265636F72645F43757272656E745F4FA0
:1030E1006666005365745F54696D65725F50726FF7
:1030F1006772616D00436C6561725F54696D6572E1
:103101005F50726F6772616D004765745F4D656EE8
:10311100755F4C616E677561676500416E6E6F75B5
:103121006E63655F4D656E755F4C616E6775616756
:103131006500436F6E74726F6C5F4465636B00531F
:10314100656C6563745F54756E65725F5365727605
:1031510069636500436F6E74726F6C5F54756E6561
:10316100720053656E645F56656E646F725F436F84
:103171006D6D616E640042726F6164636173745F4F
:1031810056656E646F725F436F6D6D616E6400565C
:10319100656E646F725F52656D6F74655F427574C1
:1031A100746F6E5F507265737365640056656E640B
:1031B1006F725F52656D6F74655F427574746F6E87
:1031C1005F52656C65617365640052657175657305
:1031D100745F4D656E7500557365725F436F6E74F4
:1031E100726F6C5F507265737365640055736572BD
:1031F1005F436F6E74726F6C5F52656C656173656E
:103201006400526571756573745F53797374656D8C
:103211005F417564696F5F4D6F64650055706461EE
:1032210074655F4465766963655F496E666F0052D8
:103231006571756573745F496D6167655F56696531
:10324100775F4F6E00526571756573745F54657871
:10325100745F566965775F4F6E00416E6E6F756E74
:1032610063655F4163746976655F536F757263650A
:10327100005365745F496E6163746976655F536F6E
:103281007572636500526571756573745F44697326
:10329100706C61795F4F53445F537472696E67005C
:1032A100496E666F726D5F4D656E755F53746174C3
:1032B1007573005365745F53797374656D5F417500
:1032C10064696F5F4D6F6465005265706F72745F02
:1032D1005265636F72645F537461747573005265F4
:1032E100706F72745F54696D65725F537461747548
:1032F10073005265706F72745F54696D65725F43DC
:103301006C65617265645F53746174757300556EA9
:10331100737570706F727465645F4D657373616707
:103321006500496D6167655F566965775F4F6E003E
:10333100546578745F566965775F4F6E00416374B9
:103341006976655F536F7572636500496E61637479
:103351006976655F536F7572636500526571756556
:10336100737465645F666F725F5374616E646279D2
:1033710000496E666F726D65645F4D656E755F4C79
:10338100616E67756167650052656365697665643D
:103391005F56656E646F725F436F6D6D616E640041
:1033A10052656365697665645F56656E646F725FC9
:1033B10052656D6F74655F427574746F6E5F5072A4
:1033C10065737365640052656365697665645F560C
:1033D100656E646F725F52656D6F74655F4275747F
:1033E100746F6E5F52656C656173656400446973E7
:1033F100706C61795F4F53445F537472696E6700FB
:10340100496E666F726D65645F4D656E755F53746D
:10341100617475730052656365697665645F5573A0
:1034210065725F436F6E74726F6C5F507265737318
:1034310065640052656365697665645F557365729D
:103441005F436F6E74726F6C5F52656C656173651B
:10345100640053797374656D5F417564696F5F4D85
:103461006F64655F536574004465766963655F49A0
:103471006E666F5F4368616E676564005365745F74
:1034810053747265616D5F50617468005265717546
:1034910065737465645F5265636F72645F437572CF
:1034A10072656E74005265717565737465645F52FF
:1034B10065636F72645F43757272656E745F4F66A8
:1034C10066005265717565737465645F5365745FF9
:1034D10054696D65725F50726F6772616D005265FC
:1034E100717565737465645F5365745F54696D6567
:1034F100725F50726F6772616D5F5469746C6500C1
:103501005265717565737465645F436C6561725F63
:1035110054696D65725F50726F6772616D005265BB
:10352100717565737465645F666F725F4D656E7505
:10353100005265717565737465645F436F6E747273
:103541006F6C5F4465636B0053656C6563746564A0
:103551005F54756E65725F5365727669636500527B
:1035610065717565737465645F436F6E74726F6CBA
:103571005F54756E6572005265717565737465642B
:103581005F666F725F53797374656D5F41756469CE
:103591006F5F4D6F646500526F7574696E675F4F41
:1035A100666600443D307825302E325820446565EA
:1035B1007020436F6C6F7220446574656374656439
:1035C1000D0A00443D307825302E32582034204FEA
:1035D100757470757420537570706F72740D0A0074
:1035E100443D307825302E325820547820545245AD
:1035F10047203D20307825302E32580D0A004552A3
:10360100524F523A204E3D307825302E32582041CB
:103611004B535620524459202D204D4355204949A2
:10362100432025640D0A004552524F523A204E3D27
:10363100307825302E325820414B53562072656127
:1036410064202D204D4355204949432025640D0A0E
:10365100004552524F523A204E3D307825302E329D
:103661005820414B53562072656164202D204B65D3
:10367100792057726F6E670D0A004552524F523AC8
:10368100204E3D307825302E325820547820526912
:103691002072656164202D204D4355204949432006
:1036A10025640D0A004552524F523A204E3D307862
:1036B10025302E325820424B5356207265616420CA
:1036C1002D20444E204444432025640D0A004552D8
:1036D100524F523A204E3D307825302E32582042FA
:1036E1004B53562072656164202D204B657920571C
:1036F100726F6E670D0A004552524F523A204E3D8D
:10370100307825302E325820527820526920726547
:103711006164202D20444E204444432025640D0A39
:10372100004552524F523A204E3D307825302E32CC
:1037310058204B5356204649464F207265616420FC
:103741002D20444E204444432025640D0A00455257
:10375100524F523A204E3D307825302E3258204B70
:103761005356204649464F2072656164202D204BF7
:1037710065792057726F6E670D0A004552524F529C
:103781003A204E3D307825302E3258204544494468
:103791002062302072656164202D20444E20444413
:1037A100432025640D0A004552524F523A204E3DA6
:1037B100307825302E3258204544494420436865ED
:1037C100636B206661696C65642C207045444944D3
:1037D1005B3132365D3D307825302E3258203E2027
:1037E100380D0A004552524F523A204E3D3078254D
:1037F100302E325820454449442062692072656167
:1038010064202D20444E204444432025640D0A00A9
:103811004552524F523A204E3D307825302E325883
:10382100204544494420636865636B73756D206569
:1038310072726F720D0A005741524E494E473A203B
:10384100443D307825302E3258204E6F204550436C
:10385100432064657465637465640A0D00443D30FA
:103861007825302E325820455043432064657465D5
:1038710063746564205665723D25642E25640A0DC6
:10388100005741524E494E473A204E6F20446576CB
:1038910069636520666F756E640D0A005741524E6B
:1038A100494E473A204E6F20417564696F20537924
:1038B1007374656D20666F756E640D0A0057415211
:1038C1004E494E473A20443D307825302E3258201B
:1038D10045504343204576656E74204D6973736985
:1038E1006E670D0A004552524F523A20443D3078DE
:1038F10025302E3258204550434320436F6D6D6172
:103901006E642054696D652D6F75740D0A00455202
:10391100524F523A20494943206661696C656420DF
:1039210025642C20494943416464723D3078253037
:103931002E32582C20526567416464723D307825DF
:10394100302E32580D0A00FF3071FF3076FF30877C
:10395100FF309BFF30A3FF30AEFF30B6FF30C2FF18
:1039610030D1FF30E4FF30F6FF310AFF311CFF3167
:1039710033FF3140FF3155FF3163FF3177FF319024
:10398100FF31ADFF31CBFF31D8FF31EDFF3203FF06
:10399100321DFF3230FF3246FF325BFF3272FF329F
:1039A10086FF32A1FF32B4FF32CAFF32DFFF32F3AA
:1039B100FF330FFF3323FF3331FF333EFF334CFF20
:1039C100335CFF3372FF3389FF33A1FF33C7FF330A
:1039D100EEFF3401FF3416FF3434FF3453FF3469F2
:1039E100FF347DFF348DFF34A6FF34C3FF34DFFF86
:1039F1003501FF351FFF3532FF3549FF3560FF3592
:043A010078FF35987D
:0C91F40001650042FC2C0000025E00003F
:106EDF0090FC54E0FBA3E0FAA3E0F9121B3FFF90F4
:106EEF00FC57E0FBA3E0FAA3E022F090FC30E4753E
:106EFF00F001121C8EFE748025F0F58274FF3EF5B2
:106F0F00837469F090FC30E475F001121C8EFE74EE
:106F1F008025F0F58274FF3EF58322F9121B3F04A2
:106F2F00FF90FCC57B00E47A007922F0A304F022E5
:106F3F00F0A3EDF0A3EBF0A3EAF0A3E9F022121B0C
:106F4F003F04FF90FC7D7B00E47A007922F0A322BE
:106F5F00F9121B3FFF90FAF3E4F0A3EFF02290FF3A
:106F6F0080F090FC0CE47B017AFF7980F0A322F98A
:106F7F00900001021B582407F9E43AFA90FC7DE4D3
:106F8F00F0A322F9121B3FFF90FD49E4F0A3042266
:106F9F007B007A00792290FC0CE4F0A322F9121BFB
:106FAF003FFFE490FD49F0A32290FC2EE090FAF50C
:106FBF00FFE4F0A3EFF022F990FC30E0FEA3E0F540
:106FCF00828E83021B58F9900002121B58FF90000B
:106FDF0003121B58FD22F9121B3FFF7B017AFF7929
:106FEF0080227961E7C4F8540FC868FF19E7C454C9
:106FFF00F048FEE42FFDEE22F9A3E0FFA3E090FCA2
:10700F000CCFF0A3EFF0222FF9EA3EFA9000041212
:10701F001B58FF900005121B58FD2290FC2EEFF01D
:10702F00E0FE2204F0A3F07D74FF22F990FCC5E48A
:10703F00F0A3222401F9E43AFA021B3F7405F0E4AD
:10704F00A3F07D757F0122E490FC30F0A3F022F9CC
:10705F00121B3F04FF2290FCB9E0FD90FAF3E4F01D
:10706F00A3EDF0A32290FC30E0FDA3E090FC7DCDDA
:10707F00F0A3EDF022A3E4F0A3E522F07BFF7A3535
:10708F0079E12290FC30E4F0740AA3F0E4A3F0A3BA
:10709F00F02290FC31E004F02290FC30E004F0226A
:1070AF0090FCFEE014FF90FCFDE02290FC30E0FE2F
:1070BF00A3E0FFC39406EE6480948022D390FC314A
:1070CF00E0940090FC30E064802290FC33E004F008
:1070DF002290FC32E004F022C390FC33E094039042
:1070EF00FC32E064809480227480F0E4A3F07DA1F0
:1070FF007F012290FC2EE0FF90FAF522C390FD82D3
:10710F00E094E890FD81E0940322E025E0FF90FCFD
:10711F0030E033FE90FC3422A3E024FDF090FC30ED
:10712F00E034FFF02204F0A3F07DA0FF2290FD4891
:10713F00E0FF7401A8070822E52225E0F52222F0DE
:09714F00A37402F07D747F01229B
:108A2C007862A60308A60208A60190FCE4E0F9A36C
:108A3C00E0FAA3E090FC34C9126F4590FC34126E3E
:108A4C00F1126FD5127A6F90FC34126EF1126FD551
:108A5C007B0212694A90FC34126EF1F9121B3FFF33
:108A6C00126F7FFD127BD690FC34126EF1F9121B43
:108A7C003FFF126F7FFD7B0112694A12AE207D0809
:108A8C007F06127A6F7B017D087F0612694A12708D
:108A9C00561270BA501FEF25E0FFEE33FE90FC34F7
:108AAC00126EF11270167B0112694A1270A17003DA
:108ABC001270A880DCE4FB7D01FF12ACE87B02E4C1
:108ACC00FD7F0112ACE87BFF7AA379F1E4FF12B5CC
:108ADC001290FD8A74FEF07BA0E4FD12AAE47BFFE9
:0E8AEC007A00794EE4FF12B5017D0102AA2B3B
:10AE200090FC34126EF1F9121B3FFF126F7FFD127E
:10AE30007BD612984190FC34126EF1F9121B3FFF41
:0CAE4000126F7FFD127A6F7F0402B59341
:10B4B60090FC34126EF1126FD5127A6F7D02E4FFA2
:03B4C60002B1A729
:10B4EF00E4FDFF12B1A790FC34126EF1126FD5027A
:02B4FF007BD6FA
:1095D20090FDA0126F4490FDA0126EF1F9ED121BE6
:1095E200A790FDA0126EF1F9900001E4121BB912CE
:1095F2006F2B7D05128BC790FC2EE07024E5226054
:109602002090FDA0126EF1126F5F7BFF7A3579A474
:1096120012A83990FDA0126EF11270424440121B42
:10962200A775220890FDA0126EF1F9121B3F126F6E
:109632002F7D07128BC790FDA0126EF1126F2A7D4B
:1096420007128BC790FC2EE0702330132090FDA0F0
:10965200126EF1126F5F7BFF7A3579C412A83990CE
:0E966200FDA0126EF11270424480121BA7226E
:0DB56D00126F7F30E6047F0180027F002214
:109B1F0090FDA3126F4490FDA3126EF1126F7E3071
:109B2F00E51F30E60820E74C126F93802690FDA3C7
:109B3F00126EF1126F92129BA0126EF1126F928041
:109B4F002B90FDA3126EF1126F7E30E60D20E724ED
:109B5F00126FADF07B067D06801790FDA3126EF19C
:109B6F00126FAC129BA0126EF1126FACF07B047DE2
:109B7F000A12A96390FDA3126EF1126F2A7D0612CD
:109B8F008BC790FDA3126EF1126F5F12708402A843
:0D9B9F0039F07B057D0A12A96390FDA32219
:10AED00090FDA6126F44ED90FDA6600A126EF1126D
:10AEE000704244208008126EF112704254DF121B2F
:0BAEF000A790FDA6126EF1F9029B1F57
:10A79E0090FDA9126F4490FDA9126EF1126F7E30DA
:10A7AE00E40830E61C126FAD800F90FDA9126EF119
:10A7BE00126F7E30E60B126F93F07B077D0612A9A7
:10A7CE006390FDA9126EF1126F2A7D06128BC7904F
:0EA7DE00FDA9126EF1126F5F12708402A8398D
:10AEFB0090FDAC126F44ED90FDAC600A126EF11236
:10AF0B00704244108008126EF112704254EF121B03
:0BAF1B00A790FDAC126EF1F902A79E9A
:10ABD00090FDAF126F4490FDAF126EF1126F7E3098
:10ABE000E60B126F93F07B057D0612A96390FDAF13
:10ABF000126EF1126F2A7D06128BC790FDAF126E96
:0AAC0000F1126F5F12708402A83990
:10AE4C0090FDB2126F4490FDB2126EF1126F7E3013
:10AE5C00E708126FADF07B03800C90FDB2126EF11F
:0CAE6C00126FACF07B017D0712A963227D
:109E4C0090FDB5126F4490FDB5126EF1126F7E301D
:109E5C00E634752208121B3F126F2F7D05128BC73B
:109E6C0090FDB5126EF1126F7E30E7057522C08041
:109E7C000A75229490FDB5126EF1F9121B3F126F08
:109E8C002F7D06128BC790FDB5126EF1F9129B1F38
:109E9C0090FDB5126EF1F912A79E90FDB5126EF100
:109EAC00126F7E30E708126F93F07B03800B90FDEE
:0F9EBC00B5126EF1126F92F0FB7D0712A96322AF
:10ADBD0090FDB8126F4490FDB8126EF1126F2A7D9E
:10ADCD0007128BC790FDB8126EF1126F7E30E70837
:10ADDD00A216821782138006A21682178211E433FF
:02ADED00FF2243
:0EB54300126F2B7D07128BC7A215E433FF2277
:10B40C00126F2B7D07128BC790FC2EE060037F011F
:07B41C0022A214E433FF2219
:0EB55100126F2B7D08128BC7A216E433FF2267
:0EB55F00126F2B7D40128BC7A210E433FF2227
:10000E00121B3FFF90FCEA126EF112703A7403F06D
:05001E007D50028BC7BC
:10B3C400121B3FFF90FC92126EF1F9A3E0FD127084
:08B3D4003BEDF07D80028BC708
:10B43A00121B3F04FF90FCF0126EF112703A74086E
:06B44A00F07D41028BC7FA
:10005600121B3FFF90FCF6126EF112703A7414F008
:050066007D60028BC764
:10B2D50090FDBB126F4490FDBB126EF1F912A601F1
:10B2E50090FDBB126EF1126FACF0FB7D0802A963F5
:10B1EE0090FDBE126F4490FDBE126EF1F912A601D3
:10B1FE0090FDBE126EF1126F92F0E4FB7D0802A973
:01B20E0063DC
:10B20F0090FDC1126F4490FDC1126EF1F912A601AB
:10B21F0090FDC1126EF1126F92F07B077D0802A9AB
:01B22F0063BB
:10B2300090FDC4126F4490FDC4126EF1F912A60184
:10B2400090FDC4126EF1126FACF07B077D0802A96D
:01B25000639A
:10B2510090FDC7126F4490FDC7126EF1F912A6015D
:10B2610090FDC7126EF1126F92F0E4FB7D0F02A9FF
:01B271006379
:10B2F50090FDCA126F4490FDCA126EF1F912A601B3
:10B3050090FDCA126EF1126FACF0FB7D0F02A963BE
:10A1980090FD63126F44A3EDF012A60190FD6312C7
:10A1A8006EF1126F2A7D09128BC73011037F0122CD
:10A1B80090FD66E0FF12A6A9E4F522FB90FC0C12C4
:10A1C8006F36A3F07D60FF127759E4F522FB90FC0F
:10A1D8000C126F5812713412775912702AC00690F7
:10A1E800FC0C126F331270FA127759D0E04F90FCC2
:0AA1F8002EF070037F02227F002288
:1000260090FDCD126F4490FDCD126EF1F912A6012E
:1000360090FDCD126EF1126F2A7D09128BC7A212A6
:04004600E433FF227E
:10B2720090FDD0126F4490FDD0126EF1F912A6012A
:10B2820090FDD0126EF1126F92F0E4FB7D0E02A9D6
:01B292006358
:10B3150090FDD3126F4490FDD3126EF1F912A60180
:10B3250090FDD3126EF1126FACF0FB7D0E02A96396
:10B2930090FDD6126F4490FDD6126EF1F912A601FD
:10B2A30090FDD6126EF1126F92F07B047D0F02A90E
:01B2B3006337
:10B2B40090FDD9126F4490FDD9126EF1F912A601D6
:10B2C40090FDD9126EF1126FACF07B047D0F02A9D0
:01B2D4006316
:10AE780090FC96126F4490FC96126EF1F912A6019E
:10AE880090FC96126EF1F9121B3FFF90FC9A126E1D
:0CAE9800F112703A7408F07D15028BC7AF
:10AA6A0090FD67126F44A3EDF012A60190FD6712E4
:10AA7A006EF1126F2A7D0F128BC790FC2EEFF060D9
:10AA8A00167BFF7A3579FF90FD6AE0126F63126FC9
:0DAA9A00B812A8397F0022A217E433FF2272
:1093EC0090FC9D126F44A3EDF012A60190FC9D120F
:1093FC006EF112705E90FCA1126EF112703A74074D
:10940C00F07D1D128BC790FC2EEFF060127BFF7A63
:10941C0036792890FCA0E0126F631271028058120A
:10942C007056A3F0A3F0F522752201E522601A9084
:10943C00FCA1126EF1126FC6552260081270D97021
:10944C00031270E012714780E21270A17003127067
:10945C00A890FC30E07004A3E0640570CB90FC3263
:10946C00E07004A3E0641460197BFF7A36795290A3
:10947C00FCA0E0FF90FAF3E4F0A3EFF012A8397F20
:05948C0000227F012217
:10AEA40090FCA4126F4490FCA4126EF1F912A60156
:10AEB40090FCA4126EF1F9121B3FFF90FCA8126ED5
:0CAEC400F112703A7405F07D10028BC78B
:10AF7C0090FDDC126F4490FDDC126EF1F912A6010B
:10AF8C0090FDDC126EF1126F2A7D0F128BC7E52239
:0AAF9C0030E1047F0180027F0022F3
:10A91D0090FCAB126F44A3EDF012A60190FCAB12AC
:10A92D006EF112705E90FCAF126EF112703A7402FD
:10A93D00F07D22128BC790FC2EEFF060167BFF7A14
:10A94D0036797B90FCAEE0126F63126FB812A839A6
:06A95D007F00227F0122B1
:10AFA60090FCB2126F4490FCB2126EF1F912A60137
:10AFB60090FCB2126EF112705E90FCB6126EF11237
:0AAFC600703A7408F07D25028BC775
:10906A0090FD6C126F4490FD6BEFF012A6A990FD73
:10907A006C126EF1F9E4121BA790FD6C126EF1F9F5
:10908A00126FA512703212775912702AC00690FD1B
:10909A006C126EF1F9126FA512704B127759D0E06B
:1090AA004F90FC2EF060127BFF7A3679A690FD6B0A
:1090BA00E0126F631271028056127056A3F0A3F089
:1090CA00752201E522601A90FD6C126EF1126FC6CC
:1090DA00552260081270D970031270E0127147802D
:1090EA00E21270A170031270A890FC30E07004A321
:1090FA00E0640570CB90FC32E07004A3E064146075
:10910A00197BFF7A3679CF90FD6BE0FF90FAF3E492
:0D911A00F0A3EFF012A8397F00227F0122A0
:10B3350012A6A975224090FC0C126F55127032129C
:0FB345007759126F9F0412704D127759AF222261
:10AFFA0090FE1DEDF012A6A9752215126F9F127010
:10B00A00321277597B017AFE791D126FA504F0A3DB
:09B01A0004F07D747F01027759F6
:10B04C0090FDDF126F4412A6A9752218126F9F1281
:10B05C00703212775990FDDF126EF1F9126FA574F0
:07B06C000812714E02775932
:10B0730090FDE2126F4412A6A9752210126F9F125F
:10B08300703212775990FDE2126EF1F9126FA574C6
:07B093000512714E0277590E
:10A2690090FD70126F4490FD6FEFF012A6A990FD5A
:10A2790070126EF1F97408121BA790FD70126EF13D
:10A28900F9126FA512703212775912702AC006900E
:10A29900FD70126EF1F9126FA5740212704D1277EA
:10A2A90059D0E04F90FC2EF060167BFF7A3679F892
:10A2B90090FD6FE0126F63126FB812A8397F002208
:03A2C9007F0122F0
:10AC440090FDE5126F4412A6A990FDE5126EF1F98C
:10AC54007441121BA790FDE5126EF1F9126FA51253
:10AC6400703212775990FDE5126EF1F9126FA574E6
:07AC74000212704D02775936
:10AC7B0090FDE8126F4412A6A990FDE8126EF1F94F
:10AC8B007420121BA790FDE8126EF1F9126FA5123A
:10AC9B00703212775990FDE8126EF1F9126FA574AC
:07ACAB001412704D027759ED
:1081340090FCFA126F4490FCF9EFF012A6A990FC9F
:10814400FDE0703B752243FB7A00792290FC0CF031
:10815400A31270321277591270AF90FCFAB5070C63
:10816400126EF1F9126FA512704B803D126EF1F987
:10817400126FA57405F0A37401F07D75FF802A12B7
:1081840070AF90FCFAB5070F126EF1F9126FA57477
:1081940005F0A37402800D126EF1F9126FA5740537
:1081A400F0A37403F07D757F0112775990FC2EEFD4
:1081B400F090FC2EE0FF60177BFF7A37792290FC69
:1081C400F9127068E4F0A3EFF012A8397F002212CC
:1081D4007056A3F0A3F0752201E522601A90FCFA10
:1081E400126EF1126FC6552260081270D970031214
:1081F40070E012714780E21270A170031270A890AF
:10820400FC30E07004A3E0640570CB90FC32E070B5
:1082140004A3E0641460327BFF7A37794F90FCF951
:10822400E0126F6312A8391270AF6F601990FCFAF4
:10823400126EF1F9E490FC0CF0A3F0A37402F07D4B
:0C824400757F011277597F00227F012214
:1073960090FCBA126F4490FCB9EFF012A6A9E490E3
:1073A600FF80F090FC0C126F75127591E490FF80CF
:1073B600F0126FEA90FC0CF0A31271341277591296
:1073C600702AC00690FCBA126EF1F9126FA51270FF
:1073D600F7127759D0E04F90FC2EF060137BFF7ABE
:1073E60037797C90FCB9E0126F631271020274B3B4
:1073F60090FCBA126EF1F990007E121B58FFD394DE
:10740600084014127065E4F0A3EFF07BFF7A377939
:10741600A812A8397F052290FCBA126EF1F99000E5
:107426007E121B5890FCBEF0E4A3F090FCBD04F065
:1074360090FCBEE0FF90FCBDE0FED39F40030274CB
:10744600CAEEC313126F6D12759190FCBDE0540124
:10745600C43333335480126F6D127134127759125C
:10746600702AC006126F711270F7127759D0E04F6A
:1074760090FC2EF090FF80E0B4022290FCBFE070FA
:107486001C04F090FCBA126EF12480F9E43AA801CB
:10749600FCAD03126FEA7E007F80121B1990FC2E52
:1074A600E0FF60177BFF7A3779E5127065E4F0A399
:1074B600EFF012A83990FC2EE0FF2290FCBDE0040C
:1074C600F002743690FCBA126EF1F9E4121BA79022
:1074D600FCBA126EF1F990000174FF121BB990000C
:1074E6000274FF121BB990000374FF121BB99000BF
:1074F6000474FF121BB990000574FF121BB99000AB
:107506000674FF121BB9900007E4121BB9E490FC45
:107516002FF0A3F0A3F090FCBFE060067E017F0091
:1075260080047E007F80C390FC31E09FEE6480F88B
:107536001270D298501A90FCBA126EF1126FC6FFF2
:1075460090FC2FE02FF01270A170CB1270A880C6AD
:1075560090FC2FE060137BFF7A38791190FCB9E03C
:10756600126F6312A8397F062290FCBFE090FCBA26
:10757600600B126EF1F990007E74018008126EF1B4
:10758600F990007EE4121BB97F002204F0A3F07D7F
:0675960060FF127759228C
:10A03B0090FDEB126F44ED121BA790FDEB126EF12E
:10A04B0012705E90FC7D126F747402F07D007C04C4
:10A05B0012895B90FC2EEFF090FDEB601C126EF101
:10A06B00126F5F7BFF7A38793812A83990FDEB12AB
:10A07B006EF1F9900001E4802B126EF1126F5F907C
:10A08B00FF80126FBB90FF81E090FAF7126FBF7BDE
:10A09B00FF7A38795E12A83990FDEB126EF1F990C8
:08A0AB0000017401121BB9222F
:1084300090FD73126F44A3EDF090FD73126EF14A3C
:108440004B700302851790FD73126EF1126F7E2040
:10845000E00302851712705690FC30126F177412E9
:10846000126F1274DE126F12740FF0126FE6127038
:10847000747D027C0112895B12705690FD76E0FFDC
:1084800090FC30E475F001121C8EFC748025F0F530
:108490008274FF3CF583EF126F1274FF126F12E4C7
:1084A000F090FC30126F177463126F127468126EC2
:1084B000F97445126F127458126F127450126F12C1
:1084C0007445126F127450126F12742D126F127461
:1084D00053126F127470126F12746C126EF97474FE
:1084E000126F127474126F127465126F127472121A
:1084F0006F12E4F090FC30126F17E4F090FC301231
:108500006F17E4F090FD73126EF1126FE512707444
:088510007D097C0112895B2248
:10A5AC0090FD77126F44A3EDF090FD77126EF14A97
:10A5BC004B604190FD77126EF1126F7E30E03512D8
:10A5CC001B3FFF7D0412A32E90FD7AE0F52290FD37
:10A5DC0077126EF1F9121B3F126F5104F07D007C63
:10A5EC000512895B90FD77126EF1F9121B3FFF7D0E
:05A5FC000312A32E2252
:10AD1E0090FCFF126F4490FCFF126EF14A4B6024C0
:10AD2E0090FCFF126EF1126F7E30E018121B3FFF87
:10AD3E0090FD02126EF1F9126F8B7402F07D077C9A
:05AD4E000112895B22E7
:107FFB0090FC54126F4490FC54126EF14A4B700378
:10800B0002811D90FC54126EF1126F7E20E0030270
:10801B00811D126EEEF9121B3F24FE607414607109
:10802B0014600D1470030280FE2404600302811D92
:10803B0090FC5A126EF1F9121B3F601DEA494B601E
:10804B001890FC54126EF1F9121B3FFF90FC5A1260
:10805B006EF1F9126F8B12811E126EDFF9126F8B9C
:10806B0004F07D09FC12895B126EDF2403126F870B
:10807B00128129126EDF2406126F8704F07D0BFC30
:10808B0012895B126EDF126F8504F07D28FC028172
:10809B001A90FC5A126EF1F9121B3F601DEA494B04
:1080AB00601890FC54126EF1F9121B3FFF90FC5AB2
:1080BB00126EF1F9126F8B12811E126EDFF9126FB5
:1080CB008B04F07D09FC12895B126EDF2403126FA7
:1080DB0087128129126EDF2406126F8704F07D0B45
:1080EB00FC12895B126EDF126F857408F07D297CA0
:1080FB0001801C126EDFF9126F8B04F07D0AFC12EB
:10810B00895B126EDF126F857402F07D317C011278
:10811B00895B22740EF07D127C0112895B22740341
:09812B00F07D0F7C0112895B223A
:10AD530090FD05126F4490FD05126EF14A4B60247D
:10AD630090FD05126EF1126F7E30E018121B3FFF4B
:10AD730090FD08126EF1F9126F8B7403F07D0C7C59
:05AD83000112895B22B2
:10A9EC0090FC6F126F4490FC6F126EF14A4B700327
:10A9FC007F012290FC6F126EF1126F7E20E0037FBC
:10AA0C000122121B3F04FF90FC72126EF1F9A3128B
:0FAA1C0070777D007C0712895B90FC2EEFF02293
:108C910090FC5D126F4490FC5D126EF14A4B7002C4
:108CA100FF2290FC5D126EF1126F7E20E0037F00C7
:108CB10022786076000876017860E6FE08E6FFC358
:108CC100940FEE94004003028D4EEF64054E606FE9
:108CD10090FC5D126EF112705EC007126FF13402EA
:108CE100FC126F5204F0D00712895BE522F4604F49
:108CF100E522604B90FC5D126EF112705EC00712AE
:108D01006FF13402FC90FC60126EF1F9126F8B74FA
:108D11000FF0D00712895B90FC5D126EF112705E4C
:108D2100C007126FF13403FC90FC63126EF1F9126B
:108D31006F8B740EF0D00712895B7861E6FF2278A1
:108D41006106E6186003028CB906028CB97BFF7AD2
:098D510038798212A8397F0F2243
:10A2CC0090FD0B126F4490FD0B126EF14A4B700215
:10A2DC00FF2290FD0B126EF1126F7E20E0037F00C7
:10A2EC0022126F4D04F07D507C0212895BE522F442
:10A2FC006024E522602090FD0B126EF112705E90CE
:10A30C00FD0E126EF1F9126F8B7409F07D507C0208
:10A31C0012895B7F05227BFF7A38799D12A8397FE1
:02A32C0000220D
:10ACB20090FD11126F4490FD11126EF14A4B602506
:10ACC20090FD11126EF1126F7E30E019121B3F04DB
:10ACD200FF90FD14126EF1F9126F8B740FF07D006C
:06ACE2007C0212895B22D6
:109FC20090FD7B126F44A3EDF090FD7B126EF14A7F
:109FD2004B605A90FD7B126EF1126F7E30E04EE4C0
:109FE20090FF80F0126FE6126F8B04F0FDFC128975
:109FF2005B90FF8074FF12709A90FD7B126EF112DB
:10A002006FE5126F8B12A0307F0112B59F90FF8017
:10A012007405F090FD7EE090FF81F0E4A3F090FDE6
:10A022007B126EF1126FE5126F8B12A03022740355
:09A03200F07D207C0112895B2203
:10AD880090FD17126F4490FD17126EF14A4B602424
:10AD980090FD17126EF1126F7E30E018121B3FFF04
:10ADA80090FD1A126EF1F9126F8B7408F07D207CF9
:05ADB8000112895B227D
:10A12A0090FC66126F44A3EDF090FC66126EF14A41
:10A13A004B605A90FC66126EF1126F7E30E04E123E
:10A14A001B3FFF7B017AFC7969126F8B04F0FDFCDF
:10A15A0012895B90FC6BE0FE602090FC66126EF147
:10A16A00F9121B3FFF90FC6C126EF1F9EEFD126FB3
:10A17A008BEDF07D007C0512895B90FC66126EF116
:0EA18A00F9121B3FFF90FC6AE0FD12A32E228B
:109CC00090FDEE126F4490FDEE126EF14A4B700261
:109CD000C32290FDEE126EF1126F7E20E002C322CD
:109CE000D390FC2DE0942090FC2CE0648094804084
:109CF0001C90FDEE126EF1126F5F7BFF7A3879BE19
:109D000012A839E490FC2CF0A3F07865F67865E6AB
:109D1000603290FDEE126EF1F9126F4D04F07D0588
:109D2000FC12895B30110F7865E6600116E490FC47
:109D30002CF0A3F0D32290FC2DE004F0700690FCF0
:069D40002CE004F0C32238
:10A32E0090FD7FEFF0ED12709990FD7FE0126F506F
:10A33E0004F07D06FC12895BEF7004E52260187F45
:10A34E000112B59F90FD82E004F0700690FD81E051
:10A35E0004F012710B40D212710B40107BFF7A3851
:10A36E0079E690FD7FE0126F6312A83990FD7FE0D1
:10A37E00FF7B017AFD7980126F8B04F07D06FC0263
:02A38E00895BE9
:10A6A90090FE1EEFF01270561270BA504274047E7A
:10A6B90000A807088005C333CE33CED8F9FF90FE32
:10A6C9001EE0FDEF5D90FC31600E127119126EF102
:10A6D900127016127A6F800C127119126EF11270C3
:10A6E90016127BD61270A170031270A802A6B102CD
:02A6F900B15B53
:10A6010090FD86EDF090FD83126F44126F2B7D0754
:10A61100128BC790FD83126EF1126F7E30E714909A
:10A62100FD86E05403FFE52254036F6026E52254C2
:10A63100FC801290FD86E05401FFE52254016F6019
:10A6410012E52254FE4FF522121B3F126F2F7D0798
:04A65100128BC7227F
:10A9630090FD48EBF090FD46EFF0A3EDF0EF126F92
:10A973002E128BC790FD49E07002A3E0600D1271A7
:10A983003C8002C333D8FC4222800C12713C80020B
:10A99300C333D8FCF4522290FD46E0FFA3E0FD123E
:05A9A3006F30028BC7BC
:108BC70090FCC0EF126F3F12709290FCC0E030E053
:108BD7002614FD7B017AFC79C1126FA5128C8712CE
:108BE700702AC00690FCC0E0FD90FCC2126EF11224
:108BF7007007E4A3F0802990FCC0E0FD7B017AFCBC
:108C070079C1126FA5128C8712702AC00690FCC01A
:108C1700E0FD90FCC2126EF1127007A37402F0E43B
:108C2700FF127759D0E04F90FC2EF090FC2EE060B9
:108C37002390FC30A3E0FF12B5931270CB948040D1
:108C4700031271271270D970031270E01270E75087
:108C570003028BD190FC2EE0FF601F7BFF7A3979EE
:108C67000F126F6490FCC0126FBB90FCC1E0FF90C5
:108C7700FAF7E4F0A3EFF012A83990FC2EE0FF22F8
:0A8C870004F0A3F0E4FF1277592275
:10895B0090FC77EFF0A3EC126F3F12709290FC77C4
:10896B00E030E02614FD7B017AFC7978126FA512BA
:10897B008A2012702AC00690FC77E0FD90FC7A12D8
:10898B006EF1127007E4A3F0802990FC77E0FD7B79
:10899B00017AFC7978126FA5128A2012702AC00610
:1089AB0090FC77E0FD90FC7A126EF1127007A374C5
:1089BB0002F0E4FF127759D0E04F90FC2EF090FCC0
:1089CB002EE0602390FC30A3E0FF12B5931270CB26
:1089DB00948040031271271270D970031270E01249
:1089EB0070E7500302896890FC2EE0FF60217BFF4B
:1089FB007A39790F126F6490FC77126FBB90FC7809
:108A0B00E0FFA3E090FAF7CFF0A3EFF012A83990B4
:108A1B00FC2EE0FF227402F0A314F0E4FF1277594E
:018A2B002228
:10A3F10090FE13EEF0A3EFF0ED30E00A785F06E691
:10A4010018703506803290FE13E07002A3E0703DB3
:10A41100786FA6B5ED540E785E760008F618E6FE64
:10A4210008E67807C333CE33CED8F9FF786FE6FD5F
:10A43100EE785EF6EF4D08F67862860308E6FA08D4
:0EA44100E6F9785EE6FE08E6126FCEF5B4226C
:04004E0078650622A9
:0C92000041FB4C0041FB540F41FB5500AA
:1071580090FD2FE0FBA3E0FAA3E02404F9E43AFA57
:10716800121B3F54FD121BA790FD2FE0FBA3E0FA72
:10717800A3E0F92290FB59EFF090FB51E0FF7E006D
:10718800785A7CFB7D017B017AFF7982121B19906A
:10719800FD32E0FBA3E0FAA3E02403F9E43AFA02A3
:1071A8001B3F90FD2FE0FBA3E0FAA3E0229000151F
:1071B800121B58FD2290001FE4F5F0121D75900077
:1071C8001602202690FB50F0740FA3F0E490FB59B0
:1071D800F090FB51E0FF7E00785A7CFB7D017B013B
:1071E8007AFF79822290001C022026740B90FC6A98
:1071F800F0E4A3F0A304F0A374FBF0A37459F02205
:10720800900009122026EA494B22EBF0A3EAF0A3EA
:10721800E9F02290FB50F0A37402F090FB54E09048
:10722800FB59F090FF82E090FB5AF02290001FE497
:10723800F5F0021D7590001FE475F001121CDCFECC
:10724800C3E5F02290FC577401F0A374FBF0A3741B
:107258005BF022900009122026021B3FE490FB52AB
:10726800F090FB5022122026900004021B58900038
:107278001902202690FD087401F0A374FBF0A37492
:107288004DF02290FB50F07401A3F090FB54E09075
:10729800FB592290FC727401F0A374FFF0A3748070
:1072A800F022121BB97B007A00790022A37401F046
:1072B800A374FBF0A3746A22900001021B5890008B
:1072C80002021B5890FF82E0FF90FB5AF07E007884
:1072D8005B7CFB7D017B017AFF798322F0A374013B
:1072E800F0E490FB59F090FDF42290FBC7F090FB7E
:1072F800C47401F0A374F9F0A374BFF090FB562294
:1073080090FB50E090FC6AF090FB51E090FC6BF031
:10731800A3740122900003021B58121BA790FD2999
:107328002290FB50F07401A3F090FF92E02254FDEC
:10733800121BA790FDF422900001E4021BB99000F3
:107348001F121CA4C322121B1990FDF422900005E1
:10735800021B5890001FE475F064121D7574072213
:10736800122026E9240122122026E9240222900074
:1073780002E4021BB9F090FF82E0240390FB51F075
:0E73880022900015021B587B017AF979BF2272
:10ADEF0090FD1D12721290FD1DE0F9A3E0FAA3E091
:10ADFF0090FB56C912721390FD20E0F9A3E0FAA35D
:10AE0F00E090FCE4C912721390FD1D127173028A57
:01AE1F002C06
:1083400090FDF112721290FDF1127173E4121BA7ED
:1083500090FDF112717312733F127376900003E473
:10836000121BB99000047440121BB9900005E4126E
:1083700072AAC003C002C00190FDF1127173900097
:10838000061220561272ADC003C002C00190FDF16A
:108390001271739000091220561272ADC003C00210
:1083A000C00190FDF112717390000C1220561272F0
:1083B000ADC003C002C00190FDF112717390000FB7
:1083C0001220561272ADC003C002C00190FDF1121E
:1083D000717390001212205690FDF112717390008B
:1083E00015ED1272AAC003C002C00190FDF1127116
:1083F000739000161220561272ADC003C002C00165
:1084000090FDF11271739000191220561272ADC0D6
:1084100003C002C00190FDF112717390001C122084
:108420005690FDF112717390001FE4F5F0021D7576
:0601F90090FB4CEFF02228
:1087AE0090FC1412721290FC1A127173C003C00264
:1087BE00C00190FC1712717390000912205690FCA4
:1087CE001D127173C003C002C00190FC17127173A9
:1087DE0090000C12205690FC1A127173EA494B60ED
:1087EE001690FC17127173C003C002C001A3127160
:1087FE007390000612205690FC1D127173EA494BBD
:10880E00601890FC17127173C003C002C00190FC77
:10881E001D12717390000612205690FC1412717383
:10882E00C003C002C001A31271739000191220562A
:10883E0090FC1A127173EA494B601890FC14127175
:10884E0073C003C002C00190FC1A1271739000161F
:10885E0012205690FC1D127173EA494B601890FC61
:10886E0014127173C003C002C00190FC1D1271730B
:07887E0090001612205622A3
:108EE90090FC2012721290FC26127173C003C0020A
:108EF900C00190FC2312717390000F12205690FC50
:108F090029127173C003C002C00190FC231271734E
:108F190090001212205690FC26127173EA494B6098
:108F29001690FC23127173C003C002C001A3127111
:108F39007390000612205690FC29127173EA494B6E
:108F4900601890FC23127173C003C002C00190FC29
:108F59002912717390000612205690FC2612717323
:108F6900EA494B601890FC20127173C003C002C01B
:108F79000190FC2612717390001612205690FC295C
:108F8900127173EA494B601890FC20127173C00387
:108F9900C002C00190FC291271739000161220566C
:018FA90022A5
:10B4C900C003C002C00190FD2612717390001C12C6
:03B4D900205622D8
:103A050090FDF412721290FDF41271731286D65065
:103A15002590FB56127173123F9C127173127276C8
:103A2500123FB21271AD24041271A31273361271D2
:103A3500737401121BA790FDF41271731272C030DA
:103A4500E61E12733F7D40128D5A90FDF41271AD42
:103A550024041271A31273361271737401121BA719
:103A650090FDF4127173121B3F14604D14607B14AA
:103A75007003023B2624FE7003023B5C24056003B1
:103A8500023C1D90FB56127173123F9C127173120A
:103A95007276123FB21271731271EDE4FD12843029
:103AA50090FDF41271731271ED7D0112A5AC90FDBC
:103AB500F41271737401023C1A90FDF412717312C1
:103AC50091274003023C1D90FDF41271731272346C
:103AD50012B4B690FDF412717312727612AE4C9058
:103AE500FDF41271737402023C1A90FDF4127173A5
:103AF50012970E502A90FDF412717312723D9419AB
:103B0500EE94005003023C1D127234127276129E1E
:103B15004C12B4EF90FDF41271737403023C1A80D9
:103B25002A90FDF412717312727612ADBDEF601B0F
:103B350090FDF412717312723D9432EE94005003AD
:103B4500023C1D1272347405023C1A90FDF4127188
:103B550073127234023C1D90FDF412717312727669
:103B650012B56DEF601490FDF41271731272761236
:103B7500B40CEF90FDF46020801290FDF412717387
:103B850012727612B40CEF90FDF4600C1271AD2434
:103B9500041271A34402800A1271AD24041271A3A8
:103BA50054FD121BA790FDF4127173127346942CE9
:103BB500E5F09401500A90001FE475F001121D28EC
:103BC50012727612ADBDEF704F90FDF41271731243
:103BD5007346942CE5F09401402E12727030E11377
:103BE50012AE2090FDF41271AD24041271A354FDA0
:103BF500121BA790FDF41271737D80128D5A90FDF2
:103C0500F41271737402800D90FDF41271AD2404E9
:103C15001271A354FD121BA790FDF412717312715A
:103C2500ED129CC04003023E6290FDF412717312C6
:103C350071ED12729BA3E4F0A37413F012A9EC903A
:103C4500FF80E0B410004003023E62903C57F82824
:103C55002873023C87023CA8023CAF023CB6023CFA
:103C6500C1023CD1023CE5023D0A023D20023D3540
:103C7500023D45023D5A023D73023D89023D9902CE
:103C85003DB81272640412737D90FF92E0B40F0880
:103C950090FB59740FF08005E490FB59F01272CC3B
:103CA500023D1512726474198017127264741A80B9
:103CB5001090FDF41271737D04023E5F12726474FC
:103CC5001C1272E41271737D40023E5F12726474BD
:103CD50006F0E4A3F090FDF41271737D40023E5F9F
:103CE500784D7CFB1271E47E007F0312734E1271D6
:103CF500731271ED12727C12AD5390FDF412717353
:103D05007D10023E5F1272647410F0A3141271D319
:103D150012734E1271737D40023E5FE490FB52F0C8
:103D250074121271CC12734E1271737D40023E5F94
:103D350012726474131272E41271737D40023E5F55
:103D4500E490FB52F0741D1271CC12734E12717314
:103D55007D40023E5F127264741EF0A37402F0E4AB
:103D650012722790FDF41271737D40023E5F12724C
:103D7500647415F074061271D212734E1271737D4C
:103D850040023E5F12726474161272E41271737D02
:103D950040023E5F90FB527401F090FB50741FF09F
:103DA500A37402F0E412722790FDF41271737D4042
:103DB500023E5F90FF8112722690FB59E064057008
:103DC50047A3E0702390FDF41271731271ED90FD1D
:103DD5000E12724F12A2CCEF6003023E6290FDF408
:103DE5001271737D80023E5F90FDF4127173127142
:103DF500ED90FD0E12724F12A2CCEF606090FDF4B3
:103E05001271737D80023E5F90FB5AE0702190FD38
:103E1500F41271731271ED90FC6012724F1272B44C
:103E2500123FA6703890FDF41271737D80802B903F
:103E3500FDF41271731271ED90FC6012724F1272E3
:103E4500B4123FA6601790FB59E0FF90FB54E0B514
:103E5500070B90FDF41271737D80129C3890FDF470
:103E65001271731272C6FD600C129C3890FDF4122B
:103E7500717312737690FDF412717312731C30E333
:103E850028E91271A154F71273381271731271ED8A
:103E9500C00374061271F5D003E4FD12A12A90FD4A
:103EA500F41271737D08029C3890FDF4127173123F
:103EB500731C30E42EE91271A154EF12733812719C
:103EC500731271ED12727C12AD5390FDF412717381
:103ED5001271EDC00390FC6A740CF0E4A3F0A30426
:103EE500023F9190FDF412717312731C30E63CE9A8
:103EF5001271A154BF121BA790FB50E0B4071A9092
:103F0500FDF41271731271ED90FD1A7401F0A37432
:103F1500FBF0A3745AF012AD8890FDF41271731280
:103F250071ED1273081271FE023F9690FDF4127145
:103F35007312731C30E517E91271A154DF1273383F
:103F45001271731271ED90FB54E0FD029FC290FD5A
:103F5500F412717312731C30E73CE91271A1547F9E
:103F6500121BA71272647418F0A37402F090FB5927
:103F750014F0E4A3F090FDF41271731271EDC00317
:103F850090FC6A7418F0A37402F0A3141271FED0A9
:103F950003E4FD12A12A2212A44F12B4B690FDF437
:103FA50022F0128C9190FB54EFF0640F2212AE4C6C
:043FB50090FDF42265
:104F9E0090FD2912721290000612202690FD2C12FE
:104FAE00721290FD2C1271AD4A4B70030253BC90DD
:104FBE00FD291271731286D6400E90FD291271735F
:104FCE001272C070030250AA90FD291271731271F1
:104FDE00C6C003C002C00190FD291271731271B5D3
:104FEE00D001D002D00312B2F590FD291271AD247A
:104FFE00041271A354FD1273221271731271C6C082
:10500E0003C002C00190FD291271731271B5D00157
:10501E00D002D00312B23090FD291271731271C6F4
:10502E00C003C002C00190FD291271731271B5D078
:10503E0001D002D0031253BD12717312727612AEEA
:10504E004C90FD291271731272341272C030E70A3D
:10505E0090FD291271737D80802190FD291271734C
:10506E001272C030E62290FD2C1271AD2401127125
:10507E00A344401273221271737D40128D5A90FD1B
:10508E00291271737402800890FD291271737401D4
:10509E00121BA790FD2912717312733F90FD2912F6
:1050AE007173121B3F14700302527214700302527A
:1050BE008B1470030252A414700302531A1470035B
:1050CE00025324240560030253571271C6C003C055
:1050DE0002C00190FD291271731271B5D001D00278
:1050EE00D0031253BD12717312727612AE4C90FD34
:1050FE002C127173121B3F704112735590FD2930A3
:10510E00E40C1271AD24051271A34410800A1271C1
:10511E00AD24051271A354EF121BA790FD2C127132
:10512E007312735590FD2930E50302521D1271ADB5
:10513E0024051271A354DF02522790FD291271AD7E
:10514E0024051271A354EF121BA754DF12732212FF
:10515E0071731271C6C003C002C00190FD29127195
:10516E00731271B5D001D002D00312B1EE90FD29A9
:10517E00127173127276129E4C90FD291271731277
:10518E0071C6C003C002C00190FD29127173127165
:10519E00B5D001D002D00312AA6AEF701090FD298B
:1051AE001271AD24051271A3441002522790FD29ED
:1051BE001271731271C6C003C002C00190FD291294
:1051CE0071731271B590FCA112729ED001D002D0F3
:1051DE00031293ECEF700F90FD291271AD2405129E
:1051EE0071A34410803390FD291271AD2405127104
:1051FE00A354EF121BA790FD29127173127389FF2E
:10520E007B017AFF798012906AEF701090FD29125F
:10521E0071AD24051271A34420021BA790FD291223
:10522E0071AD24051271A354DF121BA790FD291234
:10523E0071731271C6C003C002C00190FD291271B4
:10524E00731271B5D001D002D00312B2D590FD29E0
:10525E0012717312727612AE4C90FD291271737424
:10526E000102535290FD29127173129127400302CD
:10527E00536090FD29127173740202535290FD29EE
:10528E0012717312970E400302536090FD29127132
:10529E0073740302535290FD2C127173121B3FD381
:1052AE009403500302536090FD291271731271C65C
:1052BE00C003C002C00190FD291271731271B5D0E6
:1052CE0001D002D00312B27290FD291271731272C4
:1052DE0076129E4C90FD291271731271C6C003C0D6
:1052EE0002C00190FD291271731271B5D001D00266
:1052FE00D00312B1EE90FD291271AD24041271A3E8
:10530E0044011273221271737404803890FD2912B5
:10531E0071737405802E90FD2C1271731272709041
:10532E00FD2930E1151271AD24041271A34402124D
:10533E00732212717312735B800A1271AD24041200
:10534E0071A354FD121BA7800990FD2912717312CF
:10535E004A6390FD29127173129DCB90FD29127133
:10536E00AD500924041271A3441080072404127155
:10537E00A354EF121BA790FD291271731272C6FD72
:10538E00600C129C3890FD2912717312737690FD89
:10539E002912717312731CFF601490FD2C12719AF6
:1053AE004F127322127173900003E4121BB9221272
:0653BE00B2D590FD29228A
:1025810090FD2F12721290000612202690FD321239
:10259100721290FD321271AD4A4B7003023070120B
:1025A1007170121B3FD39401500302267A1271C637
:1025B100C003C002C0011271701271B5D001D00206
:1025C100D00312A198EF601112717012727020E5A0
:1025D100081272C0700302267A1271701271C6C09D
:1025E10003C002C0011271701271B5D001D002D0C6
:1025F1000312B2F51271581271C6C003C002C001B4
:102601001271701271B5D001D002D00312B2301222
:1026110071701271C6C003C002C0011271701271D3
:10262100B5D001D002D00312B2D51271701272343A
:102631001272C030E72B1271701271C6C003C00252
:10264100C0011271701271B5D001D002D00312A174
:1026510098EF90FD2F6005127173800E12717380D7
:102661000D1271701272C030E6047402800274019E
:10267100121BA712717012733F127170121B3FB4BB
:1026810007004003022B9090268FF828287302261A
:10269100A40227D00229B90229D1022A23022A4100
:1026A100022B211271C6C003C002C0011271701247
:1026B10071B5D001D002D00312B2D590FD321271A2
:1026C10073121B3F704B12735590FD2F30E40C12A7
:1026D10071AD24051271A34410800A1271AD240555
:1026E1001271A354EF121BA790FD32127173127372
:1026F1005590FD2F30E50D1271AD24051271A344E3
:10270100200227941271AD24051271A354DF022710
:10271100941271AA24051271A354EF121BA754DF5E
:1027210012716D1271C6C003C002C0011271701224
:1027310071B5D001D002D00312B1EE1271701271D5
:10274100C6C003C002C0011271701271B5D001D0B0
:1027510002D00312AA6AEF700C1271AA2405127139
:10276100A34410802E1271701271C6C003C002C042
:10277100011271701271B590FCA112729ED001D03C
:1027810002D0031293ECEF700D1271AA240512719D
:10279100A34410021BA71271AA24051271A354EFBE
:1027A100121BA71271701271C6C003C002C00112C0
:1027B10071701271B5D001D002D00312B2D512716D
:1027C100701271ED7D04128430127170022C251289
:1027D10071701271C6C003C002C001127170127112
:1027E100B5D001D002D00312A19890FB53EFF07045
:1027F10003022C3212717012727030E503022C3216
:1028010012723D940AEE94005003022C3290FB5355
:10281100E0B402181273469464E5F0940050030288
:102821002C32E924041271A3547F800A1271AA2464
:10283100041271A34480121BA7127170127389FFD5
:1028410012738F127396EF601B127170127346949C
:1028510019E5F094005003022C32E924051271A30A
:102861004440800A1271AA24051271A354BF121B9D
:10287100A712717012723412738F129A91EF90FD38
:102881002F60551271AD24041271A34401121BA7CC
:1028910012738F90FD457484F07D60129F497E0014
:1028A10074C32FF9EE34F9FA90FD02740112721318
:1028B1001271701271ED12AD1E1271701271ED7DF7
:1028C1000212A5AC1271701271EDC0031271F3D036
:1028D10003E4FD12A12A800D1271AD24041271A32B
:1028E10054FE121BA712717012727030E01A12712D
:1028F100C6C003C002C0011271701271B5D001D0FF
:1029010002D00312B272801B1271701271C6C00321
:10291100C002C0011271701271B5D001D002D00392
:1029210012B3151271701271EDE94A4B60381271D0
:10293100701271ED1272C030E02C1271701271C6FA
:1029410012B56DEF600D12717012727030E6047F76
:102951000180027F00EF44041272F21271731202BD
:1029610080EF604F803D1271701271C612B56DEF2C
:10297100600D12717012727030E6047F0180027F67
:1029810000127170127389FE90FB4CE0B506047E53
:102991000280027E00EE4F1272F2127173120280F7
:1029A100EF601090FD321271AD24011271A3444009
:1029B100121BA7127170801312717012723D940A6A
:1029C100EE94005003022C321272347403022C274D
:1029D10090FD32127173121B3FD394035003022CEA
:1029E100321271701271C6C003C002C0011271703F
:1029F1001271B5D001D002D00312B1EE1271701272
:102A010071C6C003C002C0011271701271B5D0014C
:102A1100D002D00312B230127170127234740402F7
:102A21002C2712717012723D9408EE94005003022B
:102A31002C321271BD12ABD01271707405022C27A9
:102A410012717012723D9496EE9400500C90FD320A
:102A510012717312727030E1441271701271BDC043
:102A610003C002C0011271701271B5D001D002D041
:102A710003120026EF70261271701271C6C003C0D6
:102A810002C0011271701271B5D001D002D00312CF
:102A9100B2D51271701272347406022C2712717041
:102AA1001271C6C003C002C0011271701271B5D09B
:102AB10001D002D00312A198EF6401703E1271702F
:102AC10012727020E72990FD2FA3A3E01271C6C0F6
:102AD10003C002C0011271701271B5D001D002D0D1
:102AE1000312B2D51271701272347401121BA71243
:102AF10071AA24041271A34480800A1271AA2404C9
:102B01001271A3547F121BA790FD321271731272BE
:102B11007020E103022C3212717012735B022C27B8
:102B210012717012723D94FAEE94005003022C322D
:102B31001271BDC003C002C0011271701271B5D013
:102B410001D002D00312B1EE12B15B127170127199
:102B5100C6C003C002C0011271701271B5D001D09C
:102B610002D003120026EF60081271707403121B69
:102B7100A71271701271C6C003C002C00112717038
:102B81001271B5D001D002D00312B2D5022C32128B
:102B910071701271C6C003C002C00112717012714E
:102BA100B5D001D002D003120026EF60201271705F
:102BB1001271C6C003C002C0011271701271B5D08A
:102BC10001D002D00312A198EF6401605E1271700E
:102BD1001271C6C003C002C0011271701271B5D06A
:102BE10001D002D00312B2F51271581271C6C0039E
:102BF100C002C0011271701271B5D001D002D003B0
:102C010012B2301271701271C6C003C002C001123B
:102C110071701271B5D001D002D00312B2D5127108
:102C2100701272347401121BA78006127170124A5D
:102C310063127170121B3FFF640C6019EFD3940291
:102C41004013EF6406600E90F9B9E020E70790F9B0
:102C5100B8E030E30AE924041271A34410800A1297
:102C610071AA24041271A354EF121BA712717012DE
:102C710071ED129CC04003022EC61271701271EDEB
:102C810012729BA3E4F0A37413F012A9EC90FF80DD
:102C9100E01220AF2CD5002D15032D20052D28067F
:102CA1002D4A072D72082D91092DAF0C2DD10D2E16
:102CB10000102E08112E1D122E2B132E46142E2B12
:102CC100152E57162E64172E71182E84192E931A4D
:102CD10000002EC690FF92E0FDB405047E01800243
:102CE1007E0090FB52EEF090FB50740112737DED6B
:102CF100B4050890FB597405F0801390FF92E0B47D
:102D01000F0890FB59740FF08004127293F0127245
:102D1100CC022D6A90FB50741BF0E4A3022DA61285
:102D210071974408022EC3784D7CFB1271E47E003A
:102D31007F03121B191271701271ED12727C12ADA8
:102D4100531271974410022EC390FB507410F0A3DC
:102D510014F090FF92E0B405047F05800590FB54C8
:102D6100E0FF90FB59EF1271D81271944440022E8A
:102D7100C390FB507412F0740F12732FB405047FCB
:102D810005800590FB54E0FF12717C4440022EC384
:102D91007413127329B405047F05800590FB54E078
:102DA100FF90FB59EFF01271974440022EC390FB44
:102DB100507415F0A37406F090FF92E0B405047FFF
:102DC10005800590FB54E0FF12717C4440022EC344
:102DD1007416127329FFB405047E05800590FB5417
:102DE100E0FE90FB59EEF01271974440121BA7EFE1
:102DF10064056003022EC61271974480022EC3122D
:102E010071974420022EC3740712728BF01271E085
:102E11007E007F081271944440022EC3740812721E
:102E21008BF01271974440022EC390FB507409F04D
:102E31007411127291F01271E07E007F1012719480
:102E41004440022EC3786A7CFB1271E47E007F0E3F
:102E5100121B19022EC6741412721B127197444070
:102E6100022EC3740D12721B1271974440022EC3BD
:102E710090FB50740EF0A374091272921271804487
:102E810040803F90FB50740F12721E1271974440A4
:102E9100803090FB507417F0A37403F090FB5974C9
:102EA1000512722A90FF84E0600790FB54E0FF80D6
:102EB100027F0090FB5BEFF01271974440121BA759
:102EC1004480121BA71271701272C630E127E924E7
:102ED100021271A354FD121BA7E490FB59F0127169
:102EE100701271ED90FC6A741AF0A37401F0A312D0
:102EF10071FE02302A1271701272C630E21DE9248D
:102F0100021271A354FB12716D1271EDC00390FC9A
:102F11006A741B1271F8D00302302A127170127296
:102F2100C630E31DE924021271A354F712716D1228
:102F310071EDC00390FC6A74061271F8D00302307F
:102F41002A1271701272C630E429E924021271A3A7
:102F510054EF12716D1271ED12727C12AD53127138
:102F6100701271EDC00390FC6A740C1271F8D003F9
:102F710002302A1271701272C630E61CE924021264
:102F810071A354BF12716D1271ED90FB52E0FD12ED
:102F910073081271FE02305D1271701272C620E761
:102FA10003023070E924021271A3547F121BA7900F
:102FB100FB59E064057042A3E0640470151271705E
:102FC1001271ED12724CA3E4F0A3F0A3F0127FFB97
:102FD100800A90FB5AE0700FA374FFF01271701217
:102FE10071ED7D0202A5AC1271701271ED12724C7D
:102FF100A3E4F0A3F0A302306C90FB5AE0640470E8
:103001002C1271701271ED12724C1272B4F0127FA7
:10301100FB1271701271ED7D0212A5AC127170126A
:1030210071EDC0031271F3D003E4FD802F90FB5AC0
:10303100E0702CA37404F01271701271ED7D041212
:1030410084301271701271ED7D0212A5AC12717093
:103051001271EDC0031271F3D003E4FD02A12A1233
:1030610071701271ED12724C1272B4F0127FFB2268
:0BB5C300E924041271A34420021BA71E
:0BB5CE00E924041271A354DF021BA744
:1086D60090FDF712721290FDF7127173121B3FD3C1
:1086E60094014003D38001C3400122127208702C0A
:1086F60090FDF712717390000C12720B701E90FDB4
:10870600F712717390000F12720B701090FDF71232
:10871600717390001212720B7002C32290FDF71251
:108726007173127208601390FDF712717312725B07
:10873600B40103D38001C340012290FDF712717387
:1087460090000C12720B601690FDF7127173900078
:108756000C12725EB40103D38001C340012290FD66
:10876600F712717390000F12720B601690FDF712DC
:10877600717390000F12725EB40103D38001C3407F
:10878600012290FDF712717390001212720B60169F
:1087960090FDF712717390001212725EB40103D34A
:0887A6008001C3400122D3222F
:1091270090FDFA12721290FDFA12717312720870A2
:109137002C90FDFA12717390000C12720B701E9036
:10914700FDFA12717390000F12720B701090FDFAF6
:1091570012717390001212720B7002D32290FDFAF3
:10916700127173127208601090FDFA127173127205
:109177005BD394014002D32290FDFA1271739000E1
:109187000C12720B601390FDFA12717390000C129F
:10919700725ED394014002D32290FDFA127173904C
:1091A700000F12720B601390FDFA12717390000F8B
:1091B70012725ED394014002D32290FDFA127173AA
:1091C70090001212720B601390FDFA1271739000E7
:0D91D7001212725ED394014002D322C32213
:10970E0090FDFD12721290FDFD12717312720860BF
:10971E001590FDFD12717312725BFF64036007EF0B
:10972E00D3940140012290FDFD12717390000C1232
:10973E00720B601890FDFD12717390000C12725E28
:10974E00FF64036007EFD3940140012290FDFD12E8
:10975E00717390000F12720B601890FDFD127173F1
:10976E0090000F12725EFF64036007EFD394014006
:10977E00012290FDFD12717390001212720B60188F
:10978E0090FDFD12717390001212725EFF64036001
:0A979E0007EFD39401400122D3220B
:109DCB0090FE0012721290FE0012717312720860F4
:109DDB001190FE0012717390000912726D20E40253
:109DEB00C32290FE0012717390000C12720B601163
:109DFB0090FE0012717390000C12726D20E402C37E
:109E0B002290FE0012717390000F12720B60119072
:109E1B00FE0012717390000F12726D20E402C322C8
:109E2B0090FE0012717390001212720B601190FE73
:109E3B000012717390001212726D20E402C322D3D0
:019E4B0022F4
:108D5A0090FE0312721290FE03127173127208606F
:108D6A002190FE0312717312725BD3940340139025
:108D7A00FE031271739000091273681271A34D12E7
:108D8A001BA790FE0312717390000C12720B6024E1
:108D9A0090FE0312717390000C12725ED39403401A
:108DAA001390FE0312717390000C1273681271A370
:108DBA004D121BA790FE0312717390000F12720BD3
:108DCA00602490FE0312717390000F12725ED394A6
:108DDA0003401390FE0312717390000F127368120E
:108DEA0071A34D121BA790FE031271739000121209
:108DFA00720B602490FE0312717390001212725E5D
:108E0A00D39403401390FE031271739000121273ED
:098E1A00681271A34D121BA7227E
:109C380090FE0612721290FE06127173127208607C
:109C48001390FE0612717390000912736F1271A3BC
:109C58004D121BA790FE0612717390000C12720B26
:109C6800601390FE0612717390000C12736F1271DC
:109C7800A34D121BA790FE0612717390000F12726B
:109C88000B601390FE0612717390000F12736F121F
:109C980071A34D121BA790FE061271739000121249
:109CA800720B601390FE0612717390001212736F9C
:089CB8001271A34D121BA7223B
:10920C00182F00000000000000000000000000000B
:0A921C000000000000000000000048
:10A6FB0085128385138222860308E6FA08E64A4B05
:10A70B002208E6FA08E6F90220D5A3E0FEA3E0FF53
:10A71B002290FFFF1220DBEFF0C2A922AA06AB07A3
:10A72B0090FE1FE025E0227C00121BEDEF22F8A625
:10A73B000308A60208A60122F8E6FE08E6FFE4FCE1
:02A74B00FD22ED
:1079040090FFFF1220DBEBF090FFFE1220DBECF087
:10791400A3EDF012A71CE58954FCFE12A6FBE0FBC4
:107924004EF5899000031220FFE044C0F58B90FED1
:1079340023E014605A1470030279DB24026003020A
:107944007A2D12A6FB12A715EE54FE7009758C163B
:10795400EEC313EF805F12A6FB12A715EE54FC7062
:1079640010758C2DEF7802CEC313CE13D8F9027A9A
:107974001C12A6FB12A715D394EAEE9415500B75AE
:107984008CFC7D1612A732027A1CAF03027A2612EF
:10799400A6FBA3E0FEEE700C758C0E12A6FBA3A34F
:1079A400E0027A1CEE54FE700F758C1D12A6FBA328
:1079B400E0C313A3E013806012A6FB12A715D394AF
:1079C400EFEE9410500A758CFE7D1112A732804898
:1079D40012A6FBE0FF804B12A6FBA3E0FEEE700BA9
:1079E400758C1012A6FBA3A3E0802DEE54FE700F3D
:1079F400758C2112A6FBA3E0C313A3E01380191214
:107A0400A6FB12A715D394EFEE94105010758CFEBC
:107A14007C007D0F121BEDEF14F58D800C12A6FB7C
:107A2400E0FF12B3547F00803CAF8C12A6FBE0FD54
:107A340025E02427F8760008A607AF8DED25E0247D
:107A440047F8760008A6077401A805088002C33326
:107A5400D8FCF5887410A805088002C333D8FC420A
:0B7A640089D2A97F019000040220DB02
:10B3540012A71C12A6FBE0FF7410A807088002C302
:0EB3640033D8FCF45289D2A99000010220DBFC
:0BB5D900EF75F003A4242F12A7392205
:0BB5E400EF75F003A4243B12A73922EE
:108E230090FE1FEFF0FBC2A9E58954FC4BF589AF17
:108E33008C786A760008A607AF8DE4FCFDFE7866A1
:108E4300121FDDEB25E0244712A7437866121FA00B
:108E5300C3EF9BFFEE9AFEED99FDEC98FCC004A9CD
:108E63000512A727242712A743D000121DA2C0046E
:108E7300C00512A7272428F9C3E7786B96FF19E7E3
:108E83001896FEE4FCFDD001D000EB2FFFEA3EFE76
:108E9300ED39FDEC38FC7866121FDD90FE23E014FB
:108EA300601C14602424027033E47F19FEFDFC78F7
:108EB30066121FA0121DA2E47B207A01801478663B
:108EC300121F94E47B0FFA80097866121F94E47BE7
:108ED30011FAF9F8121E2D7866121FDDD2A97868EF
:068EE300E6FE08E6FF2296
:03000B000285FD6E
:1085FD00C0E0C0F0C083C082C0D075D000C000C044
:10860D0001C002C003C004C005C006C007308812F7
:10861D00782F12A7026005782F12A70C758801021A
:10862D0086BB308912783212A7026005783212A704
:10863D000C7588020286BB308A12783512A702604B
:10864D0005783512A70C7588040286BB308B11781E
:10865D003812A7026005783812A70C758808804E6D
:10866D00308C11783B12A7026005783B12A70C7570
:10867D008810803A308D11783E12A7026005783E41
:10868D0012A70C7588208026308E11784112A70212
:10869D006005784112A70C7588408012308F0F78D5
:1086AD004412A7026005784412A70C758880D00784
:1086BD00D006D005D004D003D002D001D000D0D048
:0986CD00D082D083D0F0D0E0325D
:08B60400E5FF5407786CF62203
:0500060012B604002207
:10B3720012B604E6FF700476098008EFB4010C7877
:0CB382006C7602786CE660031680F822FE
:10B1CB0012B604E6FF7004760C800FEFB40106781C
:10B1DB006C76048005EFB4020922786CE6600316E6
:03B1EB0080F822C7
:10B15B0012B604E6FF700476178012EFB40106787E
:10B16B006C76098008EFB4020C786C7602786CE68A
:06B17B0060031680F822BB
:10A7EC0090FE23E014601314602624027036E5FFFB
:10A7FC0054077038786C760D802AE5FF5407146086
:10A80C0009047028786C7615801A786C760380149D
:10A81C00E5FF5407146009047012786C761A8004F2
:0DA82C00786C7605786CE660031680F822E3
:109ECB0090FE23E014602714604424027067E5FFC2
:109EDB00540714600D14601024027061786C764581
:109EEB008053786C761B804D786C76058047E5FF48
:109EFB00540714600D14601024027041786C765F67
:109F0B008033786C7628802D786C760C8027E5FF73
:109F1B0054071460101460131460162403701E7819
:109F2B006C766D8010786C762F800A786C760F804B
:0E9F3B0004E4786CF6786CE660031680F82279
:10984100303104D2AED2BE90FE23E01460301460F9
:109851005624027079E5FF54071460101460131444
:10986100601624037070786C767E8062786C76372F
:10987100805C786C76138056786C76018050E5FFB9
:109881005407146010146013146016240370477891
:109891006C76A98039786C764C8033786C761E8032
:1098A1002D786C76078027E5FF540714601014604B
:1098B100131460162403701E786C76C08010786CC7
:1098C1007658800A786C76248004786C760A786CF5
:0798D100E660031680F82297
:107D3D00303104D2AED2BE90FE23E01460781470C0
:107D4D0003027E2D24026003027E8CE5FF5407B4EE
:107D5D0007004003027E9C907D6BF8282873027DFE
:107D6D0080027D87027D91027D9B027DA5027DAF04
:107D7D00027DB9786D7603027E1F786D76010876E7
:107D8D0084027E8C786D76000876BC027E8C786DD0
:107D9D007600087658027E8C786D7600087626027D
:107DAD007E8C786D760008760D027E8C786D76006F
:107DBD00087601027E8CE5FF5407B40700400302EC
:107DCD007E9C907DD6F8282873027DEB027DF5020E
:107DDD007DFF027E09027E12027E1B027E24786DDB
:107DED007604087607027E8C786D76010876FD02A2
:107DFD007E8C786D76000876F9027E8C786D760033
:107E0D00087676807A786D76000876358071786D93
:107E1D0076000876158068786D7600087604805FA8
:107E2D00E5FF5407B407005066907E3DF82828738F
:107E3D00027E52027E5B027E64027E6A027E7302C5
:107E4D007E7C027E85786D76040876898031786D2A
:107E5D00760208763E8028786D76018016786D76EC
:107E6D00000876878019786D760008763D80107849
:107E7D006D76000876198007786D7600087606789D
:107E8D006EE61846600908E6161870F31680F022A3
:10B52300786C760A786CE6166005127D3D80F5220C
:10B53300786C7664786CE6166005127D3D80F522A2
:0CB58700AE071FEE600512984180F5220F
:0CB59300AE071FEE6005127D3D80F52222
:0CB59F00AE071FEE600512B52380F522F8
:0CB5AB00AE071FEE600512B53380F522DC
:109226000F4F0000000000000000000000000000DA
:019236000037
:10AFD00090FFFF1220DBEFF085128385138222861B
:10AFE0000308E6FA08E64A4B2208E6FA08E6F90200
:0AAFF00020D5E0FF7401A807082235
:10AA2B0090FFFF1220DBEDF012AFD012AFF28002DD
:10AA3B00C333D8FC12AFD8F0E0FF42F312AFD8A368
:10AA4B00E06005EF42F4800712AFD8E0F452F41245
:0FAA5B00AFD8E0F5F6D2A842F59000020220DB5A
:10B3AA0012AFD012AFF28002C333D8FC12AFD8F07A
:0AB3BA00E055F2FF9000010220DBD5
:10B4500012AFD012AFF28002C333D8FCF452F59091
:05B4600000010220DBE9
:10B50100EF75F003A4244FF8A60308A60208A601CC
:01B511002217
:0300030002953231
:10953200C0E0C0F0C083C082C0D075D000C000C0FF
:1095420001C002C003C004C005C006C007E5F5554E
:10955200F6F523301811784F12AFDF6005784F12FD
:10956200AFE975F601804E301911785212AFDF6003
:1095720005785212AFE975F602803A301A11785521
:1095820012AFDF6005785512AFE975F60480263018
:109592001B11785812AFDF6005785812AFE975F6E3
:1095A200088012301C0F785B12AFDF6005785B1207
:1095B200AFE975F610D007D006D005D004D003D09D
:1095C20002D001D000D0D0D082D083D0F0D0E0320F
:08923700061400000000000015
:109A000075BC01C390FC12E094A890FC11E0946135
:109A100022781408E6FA08E6F5828A830220D978CB
:109A200014860308E6FA08E64A4B2290FC0CE0FE96
:109A3000A3E0FF90FC0FE0FCA3E0FDC39FEC9E229F
:109A4000F5B7E490FC11F0A3F022E5BC540690FCBD
:109A500013F022ED5401C4333354C022781C08069D
:109A6000E6188606222415F582E434FEF58322905A
:109A7000FC11E004F02290FC137403F022E490FC4B
:109A80000FF0A3F02290FC09E0FBA3E0FAA3E0F9B9
:019A900022B3
:10ACE800EF6019D2BAED6006D2B6D2B78004D2B4FA
:10ACF800D2B543BB04E490FE16F08017D2B9ED60DC
:10AD080006D2B2D2B38004D2B0D2B143BB02E4902F
:06AD1800FE15F002AF265B
:10AF2600EF600543BB01800353BBFEEDB4020CEB9F
:10AF36005403C454F0FF129A53800C129A5344805F
:0BAF4600FFEB5403C454F04FF5B7229A
:10AAE40090FD89EBF0EF6014D2BAED6006D2B6D2D5
:10AAF400B78004D2B4D2B543BB048012D2B9ED609E
:10AB040006D2B2D2B38004D2B0D2B143BB0212B1E6
:0CAB1400A790FD89E0F5B3A3E0F5B622A0
:10B1A700E5BB54FE4FF5BBEDB40208129A54442E8A
:10B1B700F5B122129A5344AEF5B175B4FF75B21FBB
:04B1C70043B101226D
:10B51200EF75F003A42414F8A60308A60208A601F6
:01B522002206
:1077590090FC07EFF0A3EDF0A3EBF0A3EAF0A3E9A7
:10776900F0129A7DA3F0A3F0A3F090FC07E0FE12BB
:107779009A65E060037F012274152E129A677401DD
:10778900F0E5BB54FE4EF5BB75BC0190FC0EE02044
:10779900E12E90FC08E0F5BDE5B754F14402129AD8
:1077A90040E5BC20E00D1278F07003129A6F129A2E
:1077B9000340EE129A005005129A4A8003129A76F3
:1077C90090FC13E060030278E190FC08E020E003FC
:1077D90002785F129A7D129A2B40030278B290FCCC
:1077E90013E060030278B2EF24FFFFEE34FFFEEDF1
:1077F900B50715ECB5061190FC0EE020E00AE5B7D7
:1078090054F1440AF5B78008E5B754F14406F5B7D1
:10781900129A42E5BC20E00D1278F07003129A6FBB
:10782900129A0340EE129A8590FC0FE0FEA3E0F550
:10783900828E83E5BF121BB9129A005005129A4A2B
:107849008003129A7690FC10E004F0700690FC0F09
:10785900E004F00277DF129A7D129A2B504B90FCCC
:1078690013E07045129A858D828C83121B58F5BEE0
:10787900E5B754F14406129A40E5BC20E00D1278B0
:10788900FA7003129A6F129A0340EE129A00500589
:10789900129A4A8003129A7690FC10E004F070065E
:1078A90090FC0FE004F002786290FC0EE020E028E2
:1078B900E5B754F1440E129A40E5BC20E00D127868
:1078C900FA7003129A6F129A0340EE129A00500549
:1078D900129A4A8003129A7690FC07E0129A65E49C
:1078E900F090FC13E0FF2212000690FC12E004F075
:0B78F9002212000690FC12E004F022B6
:03004B0002929688
:10929600C0E0C0F0C083C082C0D075D000C000C09E
:1092A60001C002C003C004C005C006C00790FE206E
:1092B600E5BBF053BBFEE5B230E119129A1F600F11
:1092C600129A5C70010614FF781AE6FD129A11755F
:1092D600B202804AE5B230E211781AE620E006448E
:1092E60001F675B20175B2048034E5B230E3107848
:1092F6001C7600087600781AA6B575B208801FE5B8
:10930600B230E01A781AE6FD30E013129A1F600BAD
:10931600129A5C70010614FF129A1175B20190FE42
:1093260020E0F5BBD007D006D005D004D003D0028C
:0F933600D001D000D0D0D082D083D0F0D0E032A0
:03005300028FAA6F
:108FAA00C0E0C0F0C083C082C0D075D000C000C08D
:108FBA0001C002C003C004C005C006C00790FE215C
:108FCA00E5BBF0E5BB54FE4401F5BBE5B230E11F59
:108FDA007817129A216013781E129A5E700106148D
:108FEA00FF781BE6FD7817129A1375B2028050E5D6
:108FFA00B230E211781BE620E0064401F675B201B0
:10900A0075B204803AE5B230E310781E760008762D
:10901A0000781BA6B575B2088025E5B230E0207845
:10902A001BE6FD30E0197817129A21600F781E129C
:10903A009A5E70010614FF7817129A1375B201909E
:10904A00FE21E0F5BBD007D006D005D004D003D06E
:10905A0002D001D000D0D0D082D083D0F0D0E0327C
:10B02300EBF0A3EAF0A3E9F02290FD5AE0FBA3E0E2
:10B03300FAA3E0F92275A102439A03439C03539BAD
:09B04300FC227B017AFF798022D6
:1094910090FD4BEEF0A3EFF0A3EDF090FE23E0146E
:1094A100600F146014240270507F007ED07D028012
:1094B1000E7F807EA97D0380067FB07E1E7D047CA9
:1094C10000E5FF5407F9F8121EDFE47B20FAF9F8F2
:1094D10012A9A8C006C00790FD4BE0FEA3E0FBAABD
:1094E10006E4F9F8D007D00612A9A8C3E49F90FDBD
:1094F1004FF074049E90FD4EF04387807598509014
:10950100FD4EE0F5BAA3E0F5AA75A101E5A1B4010C
:109511000512B03880037595037E007F127D007BB4
:10952100017AFB79F512245B90FD4DE06002D2AC2B
:019531002217
:10A74D0090FD5012B023A3ECF0A3EDF0E4FFFE75E5
:10A75D00A101E5A1B4010512B0388003759503D3AD
:10A76D0090FD54E09FEE6480F890FD53E064809876
:10A77D00401E90FD5012B02F8F828E83121B58F504
:10A78D0099E59830E1FB5398FD0FBF00010E80CF86
:01A79D002299
:10B3DC0090FE22EFF07B017AFE79227D017C001237
:08B3EC00A74D90FE22E0FF22B4
:10AB200090FD5512B023E4A3F0A3F090FD5512B0B0
:10AB30002FA3E0FEA3E0F5828E83121B58FF601363
:10AB400012B3DC90FD59E004F070E090FD58E00491
:0CAB5000F080D890FD58E0FEA3E0FF224A
:10A8390090FAF012B02390FB1B7401F0A374FAF0A4
:10A84900A374F3F090FAF0E0F9A3E0FAA3E090FD25
:10A859003BC912B02490FB1BE0F9A3E0FAA3E090F6
:10A86900FD3EC912B02412B04512A8D312B0451248
:0DA87900B465AC06AD0712B04512A74D2224
:0300230002A655DD
:10A65500C0E0C083C082C0D075D000C004C005C0B2
:10A6650007E59830E02F90FC05E0FF2401FDE43379
:10A67500FCA3E06D7001EC601974F52FF582E434EC
:10A68500FBF583E599F090FC05E004F0E0B41002D9
:10A69500E4F05398FED007D005D004D0D0D082D0B6
:04A6A50083D0E0324C
:10B09A007FFF90FC06E0FE90FC05E06E601874F5F8
:10B0AA002EF582E434FBF583E0FF90FC06E004F021
:07B0BA00E0B41002E4F022F3
:10A5000090FD5A12B023A3ECF0A3EDF0E4FDFCD3D0
:10A5100090FD5EE09DEC6480F890FD5DE0648098C5
:10A52000402F12B09AEFF460F912B02C8D828C8318
:10A53000EF121BB9EFB40A12ED1D70011C12B02C02
:10A540008D828C83E4121BB980070DBD00010C8045
:06A55000BEAE04AF0522BF
:10923F004DFBE6000000FF000000000000F0E00022
:10924F0041FBE20041FBE30041FBF30041FBF40073
:08925F0041FBE50041FBE100C9
:109D4600C454F0FEEF4EFFF090FE09E024E6F582E3
:109D5600E434FBF58322E0FF90FE0AE022E0FE9069
:109D6600FE1CE022E090FE18FEE033333354F82266
:109D760075A101E5A1640122E090FE0AFEE0C4544B
:109D8600F0FD22E0FD90FE1CE0FCED6C22E0FF24DD
:109D9600FB24FB22C454F0FD90FBE1E05DFDEE22C6
:109DA60090FE1CE0FFEE6F2290FE0AE0540FF0A337
:109DB600E0FF22E0FEC454F05FFFEE4FF022F4FE17
:059DC600EF5EF0EE224B
:10694A0090FE0AEDF0A3EBF090FE09EFF014604917
:10695A001460791470030269FC147003026A1B2420
:10696A00FA7003026A4E147003026A95240B6003DC
:10697A00026AFC90FE0BE0FF700790FE0AE042FC00
:10698A0022EF90FE0AB40205E042C88004E0F45205
:10699A00C890FE0AE0F452FC2290FE0BE0FF70075A
:1069AA0090FE0AE042FD22EF90FBE2B40212129D31
:1069BA005CFEEF4EFF90FBE2129D4DE05F42FD222E
:1069CA00129D5C90FBE2129DC452FD2290FE0BE0E8
:1069DA00FF700790FE0AE042FE22EF90FE0AB40220
:1069EA0005E042D88004E0F452D890FE0AE0F4525E
:1069FA00FE2290FE0BE07012129D4EC083C08212DE
:106A0A009D5CFEEF4ED082D083F0129D4EE0F5B031
:106A1A002290FE0BE0FF700790FE0AE042F322EF9D
:106A2A0090FBE3B40212129D5CFEEF4EFF90FBE373
:106A3A00129D4DE05F42F322129D5C90FBE3129D92
:106A4A00C452F322129DAE7013129D4EC083C082AF
:106A5A00129D7EEE4DD082D083F08028EF90FBF31A
:106A6A00B4020E129D5C90FBF3129D46129DB980F2
:106A7A0013129D5CC454F0F4FEEF5E90FBF3129D7A
:106A8A004DE05EF0129D4EE0F58A2290FE0AE05437
:106A9A001CF0A3E0FF7018129D4EC083C082E090E4
:106AAA00FE0A129D6EFDEE4DD082D083F0803CEF3F
:106ABA0090FBF4B40220129D5C33333354F8FEEF9A
:106ACA004EFF90FBF4129D4DE0FE33333354F85FD2
:106ADA00FFEE4FF08015129D5C33333354F8F4FE09
:106AEA00EF5E90FBF4129D4DE05EF0129D4EE0F5D4
:106AFA00C122129D76706E90FE09129D9350072452
:106B0A00FE602C026C2512B18190FE0BE0FF70072B
:106B1A0090FE0AE0429B22EF90FE0AB40205E04290
:106B2A009C8004E0F4529C90FE0AE0F4529B22906E
:106B3A00FE0BE0FF700790FE0AE0429722EF90FBFF
:106B4A00E5B40212129D5CFEEF4EFF90FBE5129D2A
:106B5A004DE05F429722129D5CF4FEEF5E90FBE5EA
:106B6A00F0EE52972290FE09E0FF24FA6033146097
:106B7A004214606124036003026C2590FE0BE0FE60
:106B8A00700790FE0AE0429B22EE90FE0AB40205CC
:106B9A00E0429C8004E0F4529C90FE0AE0F4529B8E
:106BAA002290FE0BE090FE0A7004E0429422E0F488
:106BBA0052942290FE0BE0701574E62F129D54C079
:106BCA0083C082129D5CFEEF4ED082D083F0129D6C
:106BDA004EE0F59522129DAE7013129D4EC083C0F1
:106BEA0082129D7EEE4DD082D083F08028EF90FBFA
:106BFA00E1B4020E129D5C90FBE1129D46129DB912
:106C0A008013129D5CC454F0F4FEEF5E90FBE11217
:0C6C1A009D4DE05EF0129D4EE0F5AD22B5
:10B18100EF24FA6011146012146013146014240483
:10B191007013E4F5A12275A1012275A1022275A106
:06B1A100032275A1042247
:1097A800AB05AA07EA14601914601B14601D146045
:1097B8001F24FA6020146022240B7023E5805BFFCD
:1097C80022E5905BFF22E5A05BFF22E5B05BFF226C
:1097D800E5F25BFF22E58A5BFF22E5C15BFF22120F
:1097E8009D767032EA24FB24FB500624FE600C8030
:1097F80047AF0212B181E59A5BFF22E58F5470FAF8
:10980800758F7090FBE4E591F0E4F58FE04591F0F9
:109818008A8FE05BFF22EA24FA600F14601114605B
:109828001324037013E59A5BFF22E5935BFF22E59F
:09983800955BFF22E5AD5BFF2208
:107A6F0090FE17EFF0A3EDF090FE17E0FF129D527E
:107A7F00E04DF0EF14602114603414603B14604249
:107A8F0024FA605414607B240B6003027B3890FE51
:107A9F0017129D51E0F5802290FE18E0FF90FBE257
:107AAF00E05F42FD90FE17129D51E0F5902290FE8F
:107ABF0017129D51E0F5A02290FE17129D51E0F58F
:107ACF00B02290FE18E0FF90FBE3E05F42F390FEE0
:107ADF0017129D51E0F5F22290FE17E0FF129D5212
:107AEF00C083C082E090FE18129D8290FBF3E05D90
:107AFF00FDEE4DD082D083F074E62F129D54E0F549
:107B0F008A2290FE17E0FF129D52C083C082129D01
:107B1F006AFD90FBF4E05DFDEE4DD082D083F074F2
:107B2F00E62F129D54E0F5C122129D76704390FE10
:107B3F0017129D93500724FE6010027BD512B1815E
:107B4F0090FE17129D51E0F59A2290FE17E0FF125A
:107B5F009D52C083C082129D6AFD90FBE5E05DFDE2
:107B6F00EE4DD082D083F074E62F129D54E0F59144
:107B7F002290FE17E0FF24FA601414601B14602299
:107B8F002403704274E62F129D54E0F59A2290FE62
:107B9F0017129D51E0F5932290FE17129D51E0F5BB
:107BAF00952290FE17E0FF129D52C083C082E0FE27
:107BBF0090FE18E0129D9A4DD082D083F074E62F7C
:077BCF00129D54E0F5AD2208
:107BD60090FE19EFF0A3EDF090FE19E0FF129D5212
:107BE600E0FEEDF4FDEE5DF0EF1460211460351457
:107BF600603C14604324FA6056146077240B6003DB
:107C0600027C9C90FE19129D51E0F5802290FE198F
:107C1600129D51E0F59090FE1AE0FF90FBE2E05FC6
:107C2600F452FD2290FE19129D51E0F5A02290FE1D
:107C360019129D51E0F5B02290FE19129D51E0F502
:107C4600F290FE1AE0FF90FBE3E05FF452F322901D
:107C5600FE19E0FF129D52E0FEF58A74E62F129D92
:107C660054C083C08290FE1AE0C454F0FF90FBF328
:107C7600027D3190FE19E0FF129D52E0FEF5C174BF
:107C8600E62F129D54C083C08290FE1A129D6FFF8C
:107C960090FBF4027D31129D76703E90FE19129D86
:107CA60093500724FE6010027D3C12B18190FE19AC
:107CB600129D51E0F59A2290FE19E0FF129D52E0C6
:107CC600FEF59174E62F129D54C083C08290FE1A71
:107CD600129D6FFF90FBE5805290FE19E0FF24FA9B
:107CE600601414601B1460222403704A74E62F1279
:107CF6009D54E0F59A2290FE19129D51E0F59322CB
:107D060090FE19129D51E0F5952290FE19E0FF12A2
:107D16009D52E0FEF5AD74E62F129D54C083C082DD
:107D260090FE1AE0C454F0FF90FBE1E05FF4FFEE32
:077D36005FD082D083F02230
:106C260090FE1CEDF090FE1BEFF0146044146076AD
:106C3600147003026CCD147003026CEE24FA700318
:106C4600026D23147003026D76240B6003026DC877
:106C560090FE1BE0FF129D52C083C082129D63FD11
:106C6600EE6DD082D083F074E62F129D54E0F5804D
:106C76002290FE1BE0FF129D52129D63FDF4FCEE76
:106C86005CF59090FBE2E05D62FD74E62F129D5488
:106C9600C083C082129DA6D082D083F090FE1B12C4
:106CA6009D51E0F5902290FE1BE0FF129D52C0839D
:106CB600C082129D63FDEE6DD082D083F074E62F04
:106CC600129D54E0F5A02290FE1BE0FF129D52C0DB
:106CD60083C082129D63FDEE6DD082D083F074E690
:106CE6002F129D54E0F5B02290FE1BE0FF129D523C
:106CF600129D63FDF4FCEE5CF5F290FBE3E05D6251
:106D0600F374E62F129D54C083C082129DA6D082D2
:106D1600D083F090FE1B129D51E0F5F22290FE1BEF
:106D2600E0FF129D52129D63F4FDEE5DF58A74E656
:106D36002F129D54C083C08290FE1CE0C454F0FF05
:106D460090FBF3E05FFFEE6FD082D083F090FE1BE6
:106D5600E0FF129D52C083C082129D63540FFDEE68
:106D66006DD082D083F074E62F129D54E0F58A220E
:106D760090FE1BE0FF129D52129D63F4FDEE5DF541
:106D8600C174E62F129D54C083C08290FE1C129DD2
:106D96006FFF90FBF4E05FFFEE6FD082D083F09040
:106DA600FE1BE0FF129D52C083C082129D63541CDD
:106DB600FDEE6DD082D083F074E62F129D54E0F57F
:106DC600C122129D76706890FE1B129D9350072477
:106DD600FE6027026EDE12B18190FE1BE0FF129D5F
:106DE60052C083C082129D63FDEE6DD082D083F0C7
:106DF60074E62F129D54E0F59A2290FE1BE0FF12D6
:106E06009D52129D63FDF4FCEE5CF59190FBE5E06E
:106E16005D629774E62F129D54C083C082129DA6B0
:106E2600D082D083F090FE1B129D51E0F591229006
:106E3600FE1BE0FF24FA602B1460461460612403F5
:106E46006003026EDE90FE1BE0FE129D52C083C000
:106E560082129D89D082D083F074E62E129D54E072
:106E6600F59A2290FE1BE0FE129D52C083C082124C
:106E76009D89D082D083F074E62E129D54E0F5935E
:106E86002290FE1BE0FE129D52C083C082129D8995
:106E9600D082D083F074E62E129D54E0F5952274CC
:106EA600E62F129D54C083C082129D63129D9A6D77
:106EB600D082D083F074E62F129D54C083C082E046
:106EC600FF90FE1CE0540FFEEF6ED082D083F09050
:096ED600FE1B129D51E0F5AD22F6
:0BB5EF007D017BFF7AFF7F40021B19EB
:10B42300C3EE940240037FFF2274002FF58274EE73
:07B433003EF583E493FF22C4
:10A5560090FE0EEDF090FE0CEEF0A3EFF0C3EE943D
:10A5660002504274806480700374FFF4703730AF19
:10A5760002D22FC2AF90FE0DE0240090FE0CE03414
:10A58600EEF5F9A3E0F5FA78C07CFF79C07E0012FB
:10A59600B5EF90FE0EE07870F67B01797012FFC081
:06A5A600302F02D2AF22AB
:10AF510074806480700374FFF4701F30AF02D22FCD
:10AF6100C2AF75F9EEE4F5FA78807CFF7980FE12C4
:0BAF7100B5EF12FF80302F02D2AF229C
:0C926700C13041FD8B0043FD8C00000075
:10B38E0090FD8CE0FBA3E0FAA3E0F9EA494B229092
:0CB39E00FD8CA3E0FAA3E0F5828A832274
:10AC0A0075A101E5A1B4011BEF24FE600C14600ECE
:10AC1A002403702375A49C801E75A4DC801975A476
:10AC2A00FC801443F580EF24FE6009240270087545
:0AAC3A00A4B8800375A4F8D2BD226F
:0CB5B70090FD8CEBF0A3EAF0A3E9F02279
:10B0C10030300CEF70037F862290FD8BE0FF2275FC
:10B0D100A101E5A1B40107EF04F5A6AFA722EF7026
:07B0E10003AFA622AFA72276
:03006B0002A0B33D
:10A0B300C0E0C0F0C083C082C0D075D000C000C073
:10A0C30001C002C003C004C005C006C007C230758A
:10A0D300A101E5A164017019F5A612B38E602AE50A
:10A0E300A530E6047F0180027F0012B39DADA780F7
:10A0F3001512B38E6013E5A530E6047F0180027F5D
:10A103000012B39D7D101220D943A580D007D0063D
:10A11300D005D004D003D002D001D000D0D0D0825B
:07A12300D083D0F0D0E03240
:0692730041FE2301C131A0
:06B61C0090FE23EFF02276
:10B3F400EF6005D231758680E5FFB430037F01220A
:08B4040075FF30D2AF7F00227A
:08B60C00303104D2AED2BE229F
:105B7F00444247434D4420537472696E6720427507
:105B8F00666665722046756C6C0D0A0025732025BC
:105B9F005820255820255820255800627573004439
:105BAF004247434D44206275733A204275733D302E
:105BBF007825302E32582C20506F72743D30782556
:105BCF00302E32582C2053706565643D3078253067
:105BDF002E32580D0A0063697200444247434D4408
:105BEF00206369723A20436F64653D307825302E0B
:105BFF0032580D0A0077723000444247434D44201B
:105C0F007772303A2049443D307825302E32582C67
:105C1F00205265673D307825302E32582C20446154
:105C2F0074613D307825302E32580D0A0072643081
:105C3F0000444247434D44207264303A2049443D6A
:105C4F00307825302E32582C205265673D3078251C
:105C5F00302E32582C20446174613D00307825304D
:105C6F002E32580D0A0074623000444247434D44AF
:105C7F00207462303A2049443D307825302E325816
:105C8F002C205265673D307825302E32582C204D10
:105C9F0061736B3D307825302E32582C204461745F
:105CAF00613D0063623000444247434D44206362CC
:105CBF00303A2049443D307825302E32582C20522E
:105CCF0065673D307825302E32582C204D61736B2F
:105CDF003D307825302E32582C20446174613D00C0
:105CEF0077723100444247434D44207772313A2056
:105CFF0049443D307825302E32582C205265673D6F
:105D0F00307825302E32582C20446174613D307824
:105D1F0025302E32580D0A00726431004442474339
:105D2F004D44207264313A2049443D307825302E5D
:105D3F0032582C205265673D307825302E32582C42
:105D4F002053697A653D307825302E32582C204407
:105D5F006174613D002852656164206E756D6265E6
:105D6F0072206578636565642061206D6178206FAE
:105D7F006620256420627974657329000D0A00205E
:105D8F0000307825302E32582C20007462310044B8
:105D9F004247434D44207462313A2049443D3078A4
:105DAF0025302E32582C205265673D307825302E05
:105DBF0032582C204D61736B3D307825302E325880
:105DCF002C20446174613D006362310044424743BB
:105DDF004D44206362313A2049443D307825302EBE
:105DEF0032582C205265673D307825302E32582C92
:105DFF00204D61736B3D307825302E32582C204466
:105E0F006174613D0077723200444247434D442034
:105E1F007772323A2049443D307825302E32582C53
:105E2F00205265673D307825302E34582C20446140
:105E3F0074613D307825302E32580D0A007264326D
:105E4F0000444247434D44207264323A2049443D56
:105E5F00307825302E32582C205265673D3078250A
:105E6F00302E34582C2053697A653D307825302EEA
:105E7F0032582C20446174613D00746232004442F8
:105E8F0047434D44207462323A2049443D307825CF
:105E9F00302E32582C205265673D307825302E3405
:105EAF00582C204D61736B3D307825302E32582C95
:105EBF0020446174613D0063623200444247434DA8
:105ECF0044206362323A2049443D307825302E32E7
:105EDF00582C205265673D307825302E34582C20B1
:105EEF004D61736B3D307825302E32582C20446134
:105EFF0074613D004552524F523A20494943206642
:105F0F0061696C65642025642C20494943416464B0
:105F1F00723D307825302E32582C205265674164FF
:0D5F2F0064723D307825302E32580D0A0086
:0892790041FBBC0041FBBA00FF
:10759C0078A87CFB7D017BFF122294EF2278A87CDB
:1075AC00FB7D017BFF122294EF22A3F090FBA1E064
:1075BC00FF90FBA4E0FCA3E090FC85FD7B017AFB33
:1075CC0079A8E4F0A304F02278A87CFB7D017BFF72
:1075DC00122294EF2278A87CFB7D017BFF1222946F
:1075EC00EF227BFF7A5D799090FBBEE024A8F582B8
:1075FC00E434FBF583E0FFE490FAF3F0A3EFF02220
:10760C0078A87CFB7D017BFF122294EF2290FBA8D3
:10761C00F090FBA1E0FF90FBA3E0FD7B017AFB79EE
:10762C00A82278A87CFB7D017BFF122294EF22908C
:10763C00FBA3E0FEA3E04EF0A3E0F022E4F0A37481
:10764C0012F07BFF7A5D796490FAF3E4F0A3741284
:10765C00F0227BFF7A5C796B90FBA8E0FF90FAF349
:10766C00E422F0A3EDF0A3EBF0A3EAF0A3E9F09091
:10767C00FBBDE4F0A3740AF0E4A3F0A3F02290FBAA
:10768C00A3E0FD90FBA5E0FB22FDE0FBA3E0FAA349
:10769C00E0F9A3E0FFA3E090FC0CCFF0A3EFF0ED3A
:1076AC0022A3F0A37401F0A322A3F0A37422F0434D
:1076BC00FF407AFF79801220D553FFBF22E0FEA352
:1076CC00E0FF90FBBDE0FCA3E0FDC39FEC9E22E03D
:1076DC00FFE490FAF5F0A3EFF022D390FBBEE09418
:1076EC000090FBBDE0940022C390FBC0E09403909B
:1076FC00FBBFE09400227BFF90FBA0E0FFA3E02205
:10770C0078A87CFB7D017BFF122294EF22E054FED3
:10771C00FD7B0190FC0CE4F0A322A3E024FDF0908F
:10772C00FBBDE034FFF02290FC0EEFF090FBBAE0D2
:10773C00FF227BFF7A5D798B2290FBA8E0FF90FB08
:0D774C00A5E02290FBA8E0FF90FBA7E02243
:1045100012B09A90FE24EFF0F470030248D3E0FF4B
:1045200090FBBCE0FE04F074A82EF582E434FBF5A9
:1045300083EFF090FBBCE0D39412400E7BFF7A5BDC
:10454000797F12A839E490FBBCF090FE24E0FF6470
:104550000A6008EF640D60030248D3E490FBBCF0EE
:1045600090FB2174FFF0A3745BF0749B1276AD7422
:10457000FFF074801276AD74FBF0A374A01276AED7
:1045800074FBF0A374A21276AE74FBF0A374A412B1
:1045900076AE74FBF0A374A6F01276271266B1E42F
:1045A00090FBABF07A5B79AA12759C701D7A5B79EF
:1045B000AE1248D990FBA1E0FF12768A12ACE890C7
:1045C000FBA1E090FBBAF00248D37A5B79E5127563
:1045D0009C703F7A5B79E9127702CF12760412A8B9
:1045E00039D23090FBA1E090FD8BF090FD8CE0FB88
:1045F000A3E0FAA3E0F9EA494B70030248D390FD27
:104600008CA3A3E0F5828A837D10E4FF1220D902F7
:1046100048D37A5C79041275A970127A5C79081211
:1046200048D912768A7F7512B57A0248D37A5C79B6
:104630003C1275A970207A5C794012770290FAF3E7
:10464000CFF0A3EFF090FBA2E0FFA3E0CF1276DE65
:1046500012A8390246887A5C79751275D470117A7D
:104660005C797912490C12768A7F6312B57A8018C8
:104670007A5C79B21275D470337A5C79B612490CCF
:1046800012768A7F5312B57A90FBA3E0FF12B4DC56
:1046900090FBA6E4F0A3EFF07BFF7A5C796B90FBD4
:1046A000A6E0FFA3E090FAF3CF0248947A5C79EF9A
:1046B0001275E170247A5C79F312493F90FBA5E012
:1046C00090FBA8F090FBA1E0FF90FBA3E090FCCC56
:1046D0001275C71298D80248D37A5D79271275E10E
:1046E00070777A5D792B12493FD390FBA5E0941245
:1046F00090FBA4E09400400612764812A83990FB83
:10470000A1E04401FFC007127622A3E0FFA3E090DE
:10471000FCCCCFF0A3EFF0D0071298D8EF600302E3
:1047200048D390FBBDF0A3F090FBA41276C95026AD
:10473000ED540F700612773E12A83990FBBEE0547C
:10474000077003124A4F1275EE124A5970DA90FB45
:10475000BDE004F080D20248637A5D799A12760C4B
:1047600070277A5D799E1249F51298D8EF6003029E
:1047700048D3127745FEEF6E127619124A42600353
:104780000248D312765E0248947A5D79D712760C8D
:1047900070287A5D79DB1249F51298D8EF60030230
:1047A00048D3127745F4FEEF5E127619124A426042
:1047B000030248D312765E0248947A5E7914127628
:1047C0002E701712763B7A5E791812497290FBA709
:1047D000E01275B61296700248D37A5E794C127662
:1047E0002E600302486912763B7A5E795012497254
:1047F000D390FBA7E0941290FBA6E0940040061231
:10480000764812A83990FBA1E04401FFC00790FB55
:10481000A4E0FCA3127625A3E0FFA3E090FC85CFE3
:10482000F0A3EFF0D007129670EF60030248D39028
:10483000FBBDF0A3F090FBA61276C95026ED540FF5
:10484000700612773E12A83990FBBEE05407700341
:10485000124A4F1275EE124A5970DA90FBBDE0040D
:10486000F080D212773E0248D07A5E798912770CB6
:10487000702912763B7A5E798D1249A5129670EFF7
:10488000705112774FFEEF6E1275B6129670EF7080
:104890004212765EF0A3EFF00248D07A5E79C6123B
:1048A000770C702F12763B7A5E79CA1249A5129660
:1048B00070EF701F12774FF4FEEF5E1275B612960E
:1048C00070EF700F7BFF7A5C796B90FBA81276011A
:1048D00012A83990FE24E0FF227BFF90FBA0E0FFAE
:1048E000A3E090FAF3CFF0A3EFF090FBA2E0FFA3D8
:1048F000E090FAF5CFF0A3EFF090FBA4E0FFA3E087
:1049000090FAF7CFF0A3EFF012A839227BFF90FBCB
:10491000A0E0FFA3E090FAF3CFF0A3EFF090FBA2AA
:10492000E0FFA3E090FAF5CFF0A3EFF090FBA4E056
:10493000FFA3E090FAF7CFF0A3EFF012A839227BA3
:10494000FF90FBA0E0FFA3E090FAF3CFF0A3EFF01D
:1049500090FBA2E0FFA3E090FAF5CFF0A3EFF09078
:10496000FBA4E0FFA3E090FAF7CFF0A3EFF012A8CA
:1049700039227BFF90FBA0E0FFA3E090FAF3CFF099
:10498000A3EFF090FBA4E0FFA3E090FAF5CFF0A333
:10499000EFF090FBA6E0FFA3E090FAF7CFF0A3EFD3
:1049A000F012A839227BFF90FBA0E0FFA3E090FA71
:1049B000F3CFF0A3EFF090FBA4E0FFA3E090FAF5B3
:1049C000CFF0A3EFF090FBA6E0FFA3E090FAF7CFC3
:1049D000F0A3EFF012A83990FBA1E04401FF90FB97
:1049E000A4E0FCA3E0FD7B017AFB79A890FC85E4C0
:1049F000F0A304F0227BFF90FBA0E0FFA3E090FA7D
:104A0000F3CFF0A3EFF090FBA2E0FFA3E090FAF564
:104A1000CFF0A3EFF090FBA4E0FFA3E090FAF7CF74
:104A2000F0A3EFF012A83990FBA1E04401FF90FB46
:104A3000A3E0FD7B017AFB79A890FCCCE4F0A30411
:104A4000F02290FCCCE4F0A304F01298D8EF227B83
:104A5000FF7A5D798E12A8392212A83990FBBEE048
:034A600004F0223D
:1098D80090FCC7EF12766E90FBBAE0FF90FCC77A57
:1098E800FC79C812771904F0A3F012775990FBBBE2
:1098F800EFF0E0FEC00690FCC7E090FCC912769538
:1099080030E0047F0080027F02127733127759D04B
:10991800E04F90FBBBF0602390FBBEE0FF12B593D5
:109928001276E6400312772690FBC0E004F070063A
:1099380090FBBFE004F01276F4409C90FBBBE0FF84
:10994800601F7BFF7A5F790312760390FCC712765B
:10995800DB90FCC8E0FF90FAF7E4F0A3EFF012A860
:079968003990FBBBE0FF2278
:1096700090FC7FEFF0A3EC12766E90FBBAE0FF90C7
:10968000FC7F7AFC79801277197402F0A314F0122F
:10969000775990FBBBEFF0E0FEC00690FC7FE090B6
:1096A000FC8212769530E0047F0080027F02127700
:1096B00033127759D0E04F90FBBBF0602390FBBE94
:1096C000E0FF12B5931276E6400312772690FBC0B6
:1096D000E004F0700690FBBFE004F01276F4409ACC
:1096E00090FBBBE0FF60217BFF7A5F79031276037A
:1096F00090FC7F1276DB90FC80E0FFA3E090FAF70D
:0E970000CFF0A3EFF012A83990FBBBE0FF22E0
:10B4DC0090FF807485F0A3EFF074711276B57871DB
:03B4EC00E6FF2256
:0DB57A0090FF80EFF0A3EDF0EB1276B5220C
:0E92810043F9B501F9BF41F9B90041F9B80050
:1088850090FD35E0FBA3E0FAA3E0F92290001FE498
:10889500F5F0121D75900015021B58E0FEA3E0FFD0
:1088A5007C007D05121BDB90F9B5E0FBA3E0FAA384
:1088B500E02FF9EA3EA801FCAD037B017AFF798040
:1088C5002290001FE4F5F0121D7590001602202677
:1088D50090F9B9E0FFC390F9BEE09F7480F890F974
:1088E500BDE06480982290001FE475F001121CDC45
:1088F500FEC3E5F02290F9B9E075F005A4FF90F903
:10890500B5E0FBA3E0FAA3E022EBF0A3EAF0A3E9CC
:10891500F022FD7401F0A374FFF0A37480F022909F
:108925000004021B587E007F05121B1990F9B9E05F
:1089350004F0227F057E00122437EF2290F9B9E07A
:108945004480F02290001FE4F5F0021D752404F91F
:06895500E43AFA021B3FA8
:104A630090FD3512890E90000612202690FD381213
:104A7300890E128885121B3F24F9B40700400302F4
:104A83004F93904A9375F003A4C58325F0C58373B0
:104A9300024AA8024B6F024D22024D78024DD10209
:104AA3004E4B024EE790FD3812888812892430E17C
:104AB300751288851288CFC003C002C00112888591
:104AC30012889AFDD001D002D00312B20F1288854A
:104AD3001288EB9464EE94005003024F9312889172
:104AE300FF1288BF12906AEF602A12888512892408
:104AF30030E0191288CFC003C002C00112888512AA
:104B0300889AFDD001D002D00312B2721288857444
:104B130008024F9012888512889AFFE4FD12AFFABB
:104B230090FD35024D5C12888512892430E01912FC
:104B330088CFC003C002C00112888512889AFDD0B5
:104B430001D002D00312B2721288851288CFC0033B
:104B5300C002C00112888512889AFDD001D002D00C
:104B63000312B2301288857405024F9012888512A1
:104B7300889AFFE4FD12AFFA12888512889A124FC1
:104B83009490FD3530E61E1288881288CFC003C08A
:104B930002C00112888512889AFDD001D002D00389
:104BA30012B293801C1288881288CFC003C002C03F
:104BB3000112888512889AFDD001D002D00312B267
:104BC300B4E490FF88F012A8867C017D00121C4299
:104BD30090FF88E02480F582E434FFF583EDF090C4
:104BE300FF88E004F0E0C3940840DB128885128854
:104BF300CFC003C002C00112888512889A90FC9A24
:104C0300128917D001D002D00312AE781288851210
:104C1300889AFF1288BF12B04C1288851288CFC0C1
:104C230003C002C00112888512889A90FCA11289E0
:104C330017D001D002D0031293ECEF7024128885B1
:104C43001288CFC003C002C00112888512889AFD62
:104C5300D001D002D00312B3151288857407024F16
:104C63009012888512889AFF1288BF12B073128837
:104C73008512889AFF1288BF12906AEF70241288F7
:104C8300851288CFC003C002C00112888512889A9A
:104C9300FDD001D002D00312B31512888574070228
:104CA3004F901288851288CFC003C002C0011288BA
:104CB3008512889AFD90FCA8128918D001D002D0E1
:104CC3000312AEA4128885900019122026E94A4BDC
:104CD300704590F9B9E0C394085039E490F9BDF0F8
:104CE300A3F01288D550181288A01289386010904A
:104CF300F9BEE004F070EB90F9BDE004F080E3123C
:104D030088D540131288FA2FF9EA35F01288BA12BF
:104D1300892A80031289411288857409024F9012EF
:104D230088851288EB9407EE94005003024F931288
:104D330088CFC003C002C00112888512889AFDD0B3
:104D430001D002D00312AF7CEF90FD35600B1288C7
:104D530088128949740A024F901288881288CFC03A
:104D630003C002C00112888512889AFDD001D002C7
:104D7300D00302B31512888512A202EF7031128894
:104D8300851288EB940AEE94005003024F93128825
:104D9300C6C003C002C00112888512889AFDD001E3
:104DA300D002D00312B3151288857407024F9012F4
:104DB3008885128891124F9490FD3530E608128849
:104DC30088740D024F90128888740B024F90E49000
:104DD300FF80F01288851288CF12B551EF700C90C6
:104DE300FF80E004F0E0C394FA40E8E490FF81F030
:104DF3001288851288CF12B551BF010C90FF81E054
:104E030004F0E0C394FA40E81288851288CFC00307
:104E1300C002C00112888512889AFDD001D002D049
:104E23000312B2511288851288CFC003C002C00199
:104E330012888512889AFDD001D002D00312B230B5
:104E4300128885740C024F9090FD3812888812895D
:104E53002430E16C1288851288EB944BEE94005059
:104E630003024F9312894912A202EF7045128885FB
:104E730012892430E2211288CFC003C002C001127C
:104E8300888512889AFDD001D002D00312B2F512A0
:104E930088857407024F9090FD3512890612895256
:104EA3004404121BA712888590001FE475F0320298
:104EB3001D7590FD3512890612895254FB024F90DD
:104EC3001288851288CFC003C002C00112888512E0
:104ED300889AFDD001D002D00312B2F512888574EE
:104EE30007024F9012888512889AFF12B33590F902
:104EF300BAEFF030E56C128885128891FF1288BFF3
:104F030012AC4490FF80E0FD20E71CA3E0FF20E308
:104F13001612888590FC8BEFF0127E9DEF602012B5
:104F23008885740B024F9090FF80E030E70312896D
:104F33004190FF81E030E30790F9B8E04408F012B4
:104F430088851288CFC003C002C0011288851288E9
:104F53009AFDD001D002D00312B3151288857407CD
:104F6300802B1288851288EB94FAEE94004021126C
:104F730088C6C003C002C00112888512889AFDD07A
:104F830001D002D00312B3151288857407121BA730
:0B4F930022FF12B33590F9BAEFF022B4
:10A2020090FCCE12890E1288CFC003C002C001900A
:10A21200FCCE12888812889AFD90FCAF7401F0A3DC
:10A2220074FCF0A374D1F0D001D002D00312A91DA6
:10A23200EF7002FF2290FCCE12888812889AFF7B70
:10A24200017AFC79D312A269EF7002FF2290FCD34B
:10A25200E0FEA3E0FF90FCD1E0B50608A3E0B5075D
:07A26200037F01227F0022AF
:107E9D0090FC8712890EA3EDF0A3E0540FFF90F92B
:107EAD00B8E0FEEFD39E40028002AF0690F9B8EF26
:107EBD00F012AAA7E490F9BBF0A3F090FC8AE0FFC2
:107ECD0090F9BBE0FCA3E0FDC39F7480F8EC6480E7
:107EDD00984003027F6390FC8712888812889AFF6E
:107EED001288BF90FCFDEDF090FC8AE090FCFEF056
:107EFD00128134EF7002FF2290F9B9E0C39408505B
:107F0D0039E490F9BDF0A3F01288D550181288A06D
:107F1D00128938601090F9BEE004F070EB90F9BD55
:107F2D00E004F080E31288D540131288FA2FF9EAA5
:107F3D0035F01288BA12892A80031289411288BF3E
:107F4D007D0512934590F9BCE004F0700690F9BBE5
:107F5D00E004F0027EC890FC8AE0701890FC871255
:107F6D00888812889AFF1288BFE490FCFDF0A30464
:107F7D00F012813490FC8AE090FF80F090FC8BE051
:107F8D0090FF81F090FC871288881288CFC003C0C3
:107F9D0002C00190FC8712888812889AFD90FCB669
:107FAD007401F0A374FFF0A37482F0D001D002D05D
:107FBD000312AFA61288BF7D0A1293451285189041
:107FCD00FC8C12890E90FC8712888812889AFF12F9
:107FDD0088BF12AC7B90FC8C128906F8AC0212881B
:0E7FED00BD7F1412893A60037F00227F0122BB
:06928F0043FAD601FFC006
:108AFA0090FAE4E0FCA3E0FDA3E0FEA3E0FF90FA15
:108B0A00E0E0F8A3E0F9A3E0FAA3E022121FE9905B
:108B1A00FC3EE0FCA3E0FDA3E0FEA3E0FF227E0012
:108B2A007F407D0090FAD6E0FBA3E0FAA3E022EBB7
:108B3A002FFFEA3EFEE93DFDE83CFC22F9A3E054A2
:108B4A000F75F004A4F58285F08322EF4BFFEE4AFD
:108B5A00FEED49FDEC48FC226FFFEA6EFEE96DFD71
:108B6A00E86CFC225FFFEA5EFEE95DFDE85CFC2240
:108B7A0090FC3AC9F0A3EAF0A3E9F07B017AFA790A
:108B8A00BF22EF6BFFEE6AFEED69FDEC68FC2290F6
:108B9A00FC3E021FE9121F5690FC3722F074C12BCB
:108BAA00F58274FA3AF5832274C02BF58274FA3A84
:0D8BBA00F58322F912245BE490FAD3F02237
:10AAA70090FABF121FF56745230190FAC3121FF5ED
:10AAB700EFCDAB8990FAC7121FF598BADCFE90FA72
:10AAC700CB121FF51032547690FACF121FF5C3D26E
:0DAAD700E1F0128B28128BBDA3F0A3F0223A
:1093450090FD8FEBF0A3EAF0A3E9F0A3EDF0FF9019
:10935500FAD5E02FF090FAD4E03400F090FD92E0D9
:10936500FF70030293EB90FAD3E0FEC374409EFEB8
:10937500C39F5004AF06800590FD92E0FF90FAD997
:10938500EFF07E00128B2EF990FAD3E0FD7C00E918
:109395002DF9EC3AA801FCAD0390FD8F128B31F944
:1093A500121B1990FAD9E0FF90FAD3E02FF090FD47
:1093B50090E48FF0121C7890FD92E0FF90FAD9E0CE
:1093C500FEC3EF9E90FD92F090FAD3E0C394404027
:1093D5008B90FAD6128B0E128B7A125F3C128B2869
:0793E500128BBD029361220F
:10851800128B2EF990FAD3E0FF04F08F8275830056
:108528007480121BB990FAD3E0FFC374409FC394C0
:10853800025007128B28F912245B90FAD4E0FEA3AC
:10854800E07803C333CE33CED8F9F0EE90FAD4F006
:10855800E0FF128B2EF990003EEF121BB990FAD56E
:10856800E090003F121BB990FAD6128B0E128B7A4C
:10857800125F3CE490FADAF0A3F0C390FADBE094DF
:108588001490FADAE0648094805066E0FEA3E0FF7D
:1085980024BFF58274FA3EF583E0FD90FF80F07405
:1085A800C22FF58274FA3EF583E0FF90FADAE0FA1A
:1085B800A3E0FB24BFF58274FA3AF583EFF074C2A6
:1085C8002BF58274FA3AF583EDF0128BB2E0FF9046
:1085D800FF80128BA6E0FE128BB2EE128BA6EFF094
:1085E80090FADBE02404F090FADAE03400F0028537
:0585F80082128B8522B8
:105F3C0090FC37EBF0A3EAF0A3E9F0121F0690FAFD
:105F4C00DC121FE9900004121F2690FAE0121FE9E0
:105F5C00900008121F2690FAE4121FE990000C1210
:105F6C001F2690FAE8121FE9900010121F2690FAD3
:105F7C00EC121FE9E490FC3DF090FC3DE0FFD39463
:105F8C004F4003026228EFC3941050030260249028
:105F9C00FC3A128B31F9A3E02408128B49121F260C
:105FAC00C00790FC3AA3A3A3E0240D128B49121F47
:105FBC00ADD007EB128B62C00790FC3A128B31F913
:105FCC00A3E02402128B49121FADD007128B8CC098
:105FDC000790FC3A128B31128B46121FADD0071270
:105FEC008B8C90FC3E128B167801121EF3C004C0F1
:105FFC0005C006C007128B19781F121ECCD003D017
:10600C0002D001D000128B55C00790FC3A128B3194
:10601C00128B46D007121F7090FC3A128B31128BE8
:10602C0046121F26128B9990FC3E128B0BFBC00064
:10603C00C001C002C00390FADC128B1C7805121E42
:10604C00F3C004C005C006C00790FADC128B1C78A4
:10605C001B121ECCD003D002D001D000128B55D015
:10606C0003D002D001D000128B39128B9990FC3DD9
:10607C00E0D394135048A3128B0BFBC000C001C09B
:10608C0002C00390FAE0128B1C121EBF90FAE812A9
:10609C008B0B128B6EC004C005C006AB07128AFABC
:1060AC00128B6ED002D001D000128B55EF2499FFC9
:1060BC00EE3479FEED3482FDEC345A0261A690FC8C
:1060CC003DE0D39427502EA3128B0BFBC000C001D4
:1060DC00C002C003128AFA128B6290FAE8128B0B80
:1060EC00128B62EF24A1FFEE34EBFEED34D9FDEC04
:1060FC00346E0261A690FC3DE0D3943B506FA3122A
:10610C008B0BFBC000C001C002C00390FAE8128ADE
:10611C00FD128B6EC004C005C006AB07A3128B1C0E
:10612C0090FAE0A3A3A3E0128B6ED002D001D000B2
:10613C00128B55C004C005C006AB0790FAE8128B51
:10614C001C90FAE4128B0B128B6ED002D001D00093
:10615C00EB4FFFEA4EFEE94DFDE84CFCEF24DCFF73
:10616C00EE34BCFEED341BFDEC348F802D90FC3EE8
:10617C00128B0BFBC000C001C002C003128AFA12C2
:10618C008B6290FAE8128B0B128B62EF24D6FFEE27
:10619C0034C1FEED3462FDEC34CAFCD003D002D025
:1061AC0001D000128B39128B99128B1990FAEC12C8
:1061BC008B0BFBEF2BFFEE3AFEED39FDEC38FC12AE
:1061CC008B9990FAE8128B1CA3121FE990FAE41237
:1061DC008B1CA3121FE990FAE0128B1C781E121E66
:1061EC00F3C004C005C006C00790FAE0128B1C78FF
:1061FC0002121ECCD003D002D001D000128B55A3BA
:10620C00121FE990FADC128B1CA3128B1690FADC8D
:10621C00121FE990FC3DE004F0025F8590FC371200
:10622C008B31F9C002C001121F0690FADC128B0BE5
:10623C00128B3AD001D002128B9F128B312404F9AD
:10624C00E43AFAC002C001121F06128B08128B3AF4
:10625C00D001D002128B9F128B312408F9E43AFA48
:10626C00C002C001121F0690FAE4128B0B128B3A7B
:10627C00D001D002128B9F128B31240CF9E43AFA24
:10628C00C002C001121F0690FAE8128B0B128B3A57
:10629C00D001D002128B9F128B312410F9E43AFA00
:1062AC00C002C001121F0690FAEC128B0B128B3A33
:0762BC00D001D002021F56C1
:03000000029BACB4
:0C9BAC00787FE4F6D8FD758171029BF310
:101A4900E709F608DFFA8046E709F208DFFA803E7F
:101A590088828C83E709F0A3DFFA8032E309F6086C
:101A6900DFFA8078E309F208DFFA807088828C83D4
:101A7900E309F0A3DFFA806489828A83E0A3F60888
:101A8900DFFA805889828A83E0A3F208DFFA804C62
:101A990080D280FA80C680D4806980F28033801039
:101AA90080A680EA809A80A880DA80E280CA8033A2
:101AB90089828A83ECFAE493A3C8C582C8CCC5831A
:101AC900CCF0A3C8C582C8CCC583CCDFE9DEE780EA
:101AD9000D89828A83E493A3F608DFF9ECFAA9F069
:101AE900EDFB2289828A83ECFAE0A3C8C582C8CCBF
:101AF900C583CCF0A3C8C582C8CCC583CCDFEADED8
:101B0900E880DB89828A83E493A3F208DFF980CC39
:101B190088F0EF60010E4E60C388F0ED2402B40432
:101B29000050B9F582EB2402B4040050AF232345D9
:061B39008223901A99734B
:101B3F00BB010689828A83E0225002E722BBFE02A4
:091B4F00E32289828A83E49322D7
:101B5800BB010CE58229F582E5833AF583E0225042
:101B680006E92582F8E622BBFE06E92582F8E2228C
:0D1B7800E58229F582E5833AF583E49322A6
:101B8500BB010989828A83F8E028F022500327F7F0
:101B950022BBFE05F8E328F3228A838982F8E493C1
:021BA5002822F4
:101BA700BB010689828A83F0225002F722BBFE011D
:021BB700F32217
:101BB900F8BB010DE58229F582E5833AF583E8F062
:101BC900225006E92582C8F622BBFE05E92582C80E
:021BD900F222F6
:101BDB00EF8DF0A4A8F0CF8CF0A428CE8DF0A42E1E
:021BEB00FE22D8
:101BED00BC000BBE0029EF8DF084FFADF022E4CCDC
:101BFD00F875F008EF2FFFEE33FEEC33FCEE9DECA5
:101C0D00984005FCEE9DFE0FD5F0E9E4CEFD22EDEA
:101C1D00F8F5F0EE8420D21CFEADF075F008EF2F34
:101C2D00FFED33FD4007985006D5F0F222C398FD25
:051C3D000FD5F0EA22C2
:101C4200C2D5EC30E709B2D5E4C39DFDE49CFCEEBD
:101C520030E715B2D5E4C39FFFE49EFE121BEDC32D
:101C6200E49DFDE49CFC8003121BED30D507C3E428
:061C72009FFFE49EFE222C
:101C7800C5F0F8A3E028F0C5F0F8E58215827002F7
:061C88001583E038F02294
:101C8E00A3F8E0C5F025F0F0E58215827002158309
:061C9E00E0C838F0E82266
:101CA400BB0110E58229F582E5833AF583E0F5F07E
:101CB400A3E0225009E92582F886F008E622BBFE5B
:101CC4000AE92582F8E2F5F008E222E5832AF583A1
:081CD400E993F5F0A3E9932266
:101CDC00BB010FF8E58229F582E5833AF583E8022A
:101CEC001C8E5011C58229F808C5F026C6F5F018CF
:101CFC00C58236C622BBFE15C58229F808E2C5F09E
:101D0C0025F0F218E2C5823582F2E58222E5832ABB
:0C1D1C00F583E993F5F0A3E993C5F022EC
:101D2800BB010DC58229C582C5833AC583021C78CB
:101D38005011C58229F808E5F026F618F5F0E58275
:101D480036F622BBFE11C58229F808E225F0F5F027
:101D5800F218E23582F222F8E58229F582E5832A33
:0D1D6800F58374019325F0F5F0E493382223
:101D7500F8BB0111E58229F582E5833AF583E8F0A0
:101D8500E5F0A3F0225009E92582C8F608A6F0225D
:0D1D9500BBFE09E92582C8F2E5F008F22244
:101DA200E88FF0A4CC8BF0A42CFCE98EF0A42CFCE0
:101DB2008AF0EDA42CFCEA8EF0A4CDA8F08BF0A45E
:101DC2002DCC3825F0FDE98FF0A42CCD35F0FCEBBD
:101DD2008EF0A4FEA9F0EB8FF0A4CFC5F02ECD3982
:0F1DE200FEE43CFCEAA42DCE35F0FDE43CFC22EF
:101DF10075F008758200EF2FFFEE33FECD33CDCCA9
:101E010033CCC58233C5829BED9AEC99E58298402B
:101E11000CF582EE9BFEED9AFDEC99FC0FD5F0D608
:101E2100E4CEFBE4CDFAE4CCF9A88222B800C1B932
:101E31000059BA002DEC8BF084CFCECDFCE5F0CB70
:101E4100F97818EF2FFFEE33FEED33FDEC33FCEBA9
:101E510033FB10D703994004EB99FB0FD8E5E4F964
:101E6100FA227818EF2FFFEE33FEED33FDEC33FC51
:101E7100C933C910D7059BE99A4007EC9BFCE99A45
:101E8100F90FD8E0E4C9FAE4CCFB2275F010EF2F8A
:101E9100FFEE33FEED33FDCC33CCC833C810D7078A
:101EA1009BEC9AE899400AED9BFDEC9AFCE899F8C5
:0E1EB1000FD5F0DAE4CDFBE4CCFAE4C8F92258
:10A9A800C2D5E830E70FB2D5E4C39BFBE49AFAE4DA
:10A9B80099F9E498F8EC30E717B2D512A9DE121E1F
:10A9C8002DE4C39BFBE49AFAE499F9E498F8800330
:10A9D800121E2D30D50DE4C39FFFE49EFEE49DFDBD
:04A9E800E49CFC22CD
:0D1EBF00CFF4CFCEF4CECDF4CDCCF4CC22B8
:101ECC00E8600FECC313FCED13FDEE13FEEF13FFF4
:031EDC00D8F12218
:101EDF00E86010ECA2E713FCED13FDEE13FEEF1319
:041EEF00FFD8F02206
:101EF300E8600FEFC333FFEE33FEED33FDEC33FC4D
:031F0300D8F122F0
:101F0600BB010789828A830224B45005E9F8021FBF
:101F160094BBFE05E9F80224C089828A830224CC98
:101F2600BB010DE58229F582E5833AF5830224B4E7
:101F36005007E92582F8021F94BBFE07E92582F8BF
:101F46000224C0E58229F582E5833AF5830224CC92
:101F5600BB010789828A83021FE95005E9F8021F3F
:0A1F6600DDBBFE05E9F802250522A7
:101F7000BB010DE58229F582E5833AF583021FE96D
:101F80005007E92582F8021FDDBBFE07E92582F82C
:041F900002250522FF
:0C1F9400E6FC08E6FD08E6FE08E6FF2279
:0D1FA000E6FB08E6F908E6FA08E6CBF822B1
:101FAD00BB010DE58229F582E5833AF5830224DC38
:101FBD005007E92582F8021FA0BBFE07E92582F82C
:101FCD000224E8E58229F582E5833AF5830224F5BA
:0C1FDD00ECF608EDF608EEF608EFF62230
:0C1FE900ECF0A3EDF0A3EEF0A3EFF0226B
:101FF500A8828583F0D083D08212200C12200C1287
:10200500200C12200CE473E493A3C583C5F0C583AB
:10201500C8C582C8F0A3C583C5F0C583C8C582C835
:012025002298
:10202600BB010DE58229F582E5833AF58302252376
:102036005007E92582F8022511BBFE07E92582F83B
:10204600022563E58229F582E5833AF58302257543
:10205600BB0120E58229F582E5833AF583D0F0D0ED
:10206600E0F8D0E0F9D0E0FAD0E0FBE8C0E0C0F05C
:1020760002255A5018E92582F8D083D082D0E0F99B
:10208600D0E0FAD0E0FBC082C08302251ABBFE185E
:10209600E92582F8D083D082D0E0F9D0E0FAD0E00A
:0920A600FBC082C08302256C22FC
:1020AF00D083D082F8E4937012740193700DA3A3C0
:1020BF0093F8740193F5828883E4737402936860D4
:0620CF00EFA3A3A380DFD4
:0620D5008A838982E47396
:1020DB00E5132582F582E5123583F583B512048568
:1020EB0082132210AF06858213F51222858213F517
:0420FB0012D2AF222C
:0D20FF00E5132582F582E5123583F5832275
:10A8860090FD931224B47810EC4D4E4F70047CA5C5
:10A896007DA5C3EC13FCED13FDEE13FEEF13FF5085
:10A8A60010EC64CCFCED644CFDEE644EFEEF64CE21
:10A8B600FFD8DF90FD93121FE9EE547FFE2290FD34
:0DA8C60093EEF0EFA3F0A374A5F0A3F02231
:10662800E508302C0104F823282421F582E434FB02
:10663800F5832290FB1E302C0390FB21E475F001BA
:1066480012252C021B3F60EAC50C7002150B14C5FD
:106658000C202C04FF02B61490FB1E74FFF5F00208
:106668002543FF02B4A2E5096006D509037F00228D
:10667800202C0F12B48EEF6008050CE50C70020593
:106688000B2290FB1E122523121B3FFF60E890FB94
:106698001EE475F00112252C80DC126678EFC0E04C
:1066A80012666AD0E040F3809DD22C8002C22C9002
:1066B800FB1E12255AE4F50AF508F50BF50C7509C9
:1066C80000C22BC229C22AC22D12663BFF7005AF39
:1066D8000A7E0022B4253012663BFF24D0B40A009B
:1066E800500C75F00AC509A42509F50980E924CFDD
:1066F800B41A00EF5002C2E5026916D22A80D8D235
:106708002980D4D22D80D0EF12666A50081266A272
:10671800EF600E80A9EFC0E0126678D0E06F609E4F
:10672800EF607412664E80A7126678EF6069E5091B
:10673800700705098003126678EF6014202D0E1289
:106748006628E475F00112252CEF121BA7D509E67F
:10675800202D040508050A80BA12666EEFC0E01203
:10676800666AD0E0500412664EE4FF202D0E1266D1
:1067780028E475F00112252CEF121BA7EF70DA2020
:106788002D040508050A808BE509600205091266D3
:10679800A212666EEF70C6302C04E412664EE50A4B
:1067A80060030266D77EFF7FFF22202D1174FFFC55
:1067B800FDFEFF126628122523121F5605080266E1
:1067C800C6D0E080D27900800A79108006790880E6
:1067D80002790AD22EE50960020509E9C0E01266CD
:1067E800A2EF60DD126678BF2D04D22B8003BF2B89
:1067F800091266A2EF60CA12666ED0E0B40A02807F
:1068080033B40802802EBF302770027408C22EC02D
:10681800E012666ED0E0BF78028003BF5816050903
:10682800D509028007D50904D22E800B741080196F
:106838007002740ABF000AEFF8E4FCFDFEFF02686C
:10684800C9C0E0EF12664ED0E0F9E4FCFDFEFFE9B6
:10685800C0E0ECC0E0EDC0E0EEC0E0EFC0E01266E2
:106868006EEFF8D0E0FFD0E0FED0E0FDD0E0FCD045
:10687800F0E8604DB461004007B47B005002C2E507
:1068880024D0503DFA24F6500724F95034240AFA4B
:10689800EAB5F000502BCFA9F0A42FFF92D5E9C597
:1068A800F0CEA4A2D53EFE92D5E9C5F0CDA4A2D5DE
:1068B8003DFD92D5E9C5F0CCA4A2D53CFCC22E8002
:0668C8008EE8C0E0202D67
:1068CE002A202E08050A302B031224A6126628123F
:1068DE002523050820290B202A0DEE8FF012248780
:1068EE008009121F568004EF121BA7D0E012664ECD
:1068FE000266C6202D101266281225230508E50B08
:10690E00850CF012248780E81220AF67905367D170
:10691E005867074C67034266DF4867D54F67D9440F
:10692E0067304367CD4967D95567B24667B2456749
:0C693E00B247670B2A69014E0000670F8A
:10210C00E3F5F009E208B5F06D606B80F3E3F5F0F0
:10211C0009E608B5F060605E80F387F009E608B563
:10212C00F054605280F487F009E208B5F04860463C
:10213C0080F488828C8387F009E0A3B5F038603690
:10214C0080F488828C8387F009E493A3B5F0276030
:10215C002580F388828C83E3F5F009E0A3B5F016B3
:10216C00601480F388828C83E3F5F009E493A3B5C3
:10217C00F004600280F2022237808580E7808E8036
:10218C00D2803C8015806C807E809B80B5808B805B
:10219C00A1804F8070803A02224D89828A83ECFAAA
:1021AC00E493F5F0A3C8C582C8CCC583CCE493A353
:1021BC00C8C582C8CCC583CCB5F070606E80E1898F
:1021CC00828A83E493F5F0A3E208B5F05E605C804C
:1021DC00F289828A83E0F5F0A3E608B5F04D604BF6
:1021EC0080F389828A83E0F5F0A3E208B5F03C60C5
:1021FC003A80F389828A83E493F5F0A3E608B5F07C
:10220C002A602880F2805D89828A83ECFAE493F557
:10221C00F0A3C8C582C8CCC583CCE0A3C8C582C80E
:10222C00CCC583CCB5F004600280E27F00F845F0A9
:10223C00600EE863F0806480D395F01F40027F014C
:10224C002289828A83ECFAE0F5F0A3C8C582C8CC57
:10225C00C583CCE0A3C8C582C8CCC583CCB5F0CBB4
:10226C0060C980E389828A83ECFAE0F5F0A3C8C5E3
:10227C0082C8CCC583CCE493A3C8C582C8CCC58323
:10228C00CCB5F0A760A580E288F0ED2402B4040080
:10229C005099F582EB2402B40400508F232345821D
:0522AC00239021857361
:10B46500E4FFFE121B3F600C0FEF70010E09E9703F
:05B47500F20A80EF2245
:1022B100E3F5F009E208B5F06BDFF58067E3F5F0CF
:1022C10009E608B5F05EDFF5805A87F009E608B542
:1022D100F052DFF6804E87F009E208B5F046DFF6EE
:1022E100804288828C8387F009E0A3B5F036DFF65F
:1022F100803288828C8387F009E493A3B5F025DFCF
:10230100F5802188828C83E3F5F009E0A3B5F01410
:10231100DFF5801088828C83E3F5F009E493A3B59F
:10232100F002DFF40223E0808780E9809080D4808E
:102331003E8015806E807E809D80B7808D80A380D9
:10234100518074803C0223EC89828A83ECFAE49305
:10235100F5F0A3C8C582C8CCC583CCE493A3C8C596
:1023610082C8CCC583CCB5F076DFE3DEE18070892D
:10237100828A83E493F5F0A3E208B5F062DFF4808A
:102381005E89828A83E0F5F0A3E608B5F051DFF5B6
:10239100804D89828A83E0F5F0A3E208B5F040DF41
:1023A100F5803C89828A83E493F5F0A3E608B5F0D1
:1023B1002EDFF4802A8002805789828A83ECFAE436
:1023C10093F5F0A3C8C582C8CCC583CCE0A3C8C52A
:1023D10082C8CCC583CCB5F006DFE4DEE280007FA5
:1023E100FFB5F0020F2240027F012289828A83EC2D
:1023F100FAE0F5F0A3C8C582C8CCC583CCE0A3C878
:10240100C582C8CCC583CCB5F0D5DFE5DEE380CF8E
:1024110089828A83ECFAE0F5F0A3C8C582C8CCC5ED
:1024210083CCE493A3C8C582C8CCC583CCB5F0AF37
:10243100DFE4DEE280A988F0EF60010E4E60ABEDD3
:102441002402B404005098F582EB2402B404005035
:0A2451008E23234582239023287375
:10245B00EF4E6012EF60010EEDBB010B89828A8398
:10246B00F0A3DFFCDEFA2289F05007F709DFFCA9A5
:0C247B00F022BBFEFCF309DFFCA9F022FC
:10A8D30090FD3BE0FFA3E0FEA3E0CF90FB7BF0A362
:10A8E300EEF0A3EFF090FD3EE0CBF0A3E0CAF0A3BF
:10A8F300E0C9F07F2290FB7EAD82AC83121B3F8DBB
:10A90300828C83F0A309E970010ADFEC90FD3EE03D
:0AA91300FBA3E0FAA3E0F9026328B9
:109BB8000253C4E493A3F8E493A34003F68001F2AC
:109BC80008DFF48029E493A3F85407240CC8C333AE
:109BD800C4540F4420C8834004F456800146F6DF7D
:109BE800E4800B01020408102040809091E4E47E98
:109BF800019360BCA3FF543F30E509541FFEE49372
:109C0800A360010ECF54C025E060A840B8E493A338
:109C1800FAE493A3F8E493A3C8C582C8CAC583CA63
:109C2800F0A3C8C582C8CAC583CADFE9DEE780BE1B
:0192950000D8
:10248700BB010A89828A83F0E5F0A3F0225006F7A0
:0F24970009A7F01922BBFE06F3E5F009F319229D
:0E24A600C3E49FFFE49EFEE49DFDE49CFC2247
:0C24B400E0FCA3E0FDA3E0FEA3E0FF229B
:0C24C000E2FC08E2FD08E2FE08E2FF2258
:1024CC00E493FC740193FD740293FE740393FF2256
:0C24DC00E0F8A3E0F9A3E0FAA3E0FB2283
:0D24E800E2FB08E2F908E2FA08E2CBF82274
:1024F500E493F8740193F9740293FA740393FB223D
:0C250500ECF208EDF208EEF208EFF22212
:09251100E6FB08E6FA08E6F922EF
:09251A00EBF608EAF608E9F622E6
:09252300E0FBA3E0FAA3E0F922B9
:10252C00F8E0FBA3A3E0F925F0F0E5821582700238
:07253C001583E0FA38F022DC
:10254300F8E0FBA3A3E025F0F9F0E5821582700221
:072553001583E038FAF022C5
:09255A00EBF0A3EAF0A3E9F02282
:09256300E2FB08E2FA08E2F922A9
:09256C00EBF208EAF208E9F222A0
:0C257500E493FB740193FA740293F922C2
:1062C300E50D247BF582E434FBF583E0050D229094
:1062D300FB7830270390FB7BE475F00112252C0239
:1062E3001B3F2020E97F2ED2208018EF540F2490EB
:1062F300D43440D4FF30240BEF24BFB41A0050032E
:106303002461FFE50E6002150E0511E5117002050B
:106313001030270E90FB78E475F00112252CEF0264
:106323001BA702B0E87403D2278003E4C227F50D4C
:1063330090FB7812255AE4F50EF510F511E50E6081
:10634300077F2012630680F5750FFFC221C220C2AA
:1063530022C223C225C226C2281262D2FF700D3088
:1063630027057F00126317AF11AE1022B4255FC259
:10637300D5C2241262D2FF24D0B40A00501A75F099
:106383000A780E30D50508B6FF0106C6A426F62006
:10639300D5047002D22380D924CFB41A00EF50045D
:1063A300C2E5D224026518D22180C6D22080C0D291
:1063B3002280BCD2D580BAD22580B47F2012630656
:1063C3002022077401B50E0040F11262C3FF12636D
:1063D30006026340D228D22680951262C3FB126262
:1063E300C3FA1262C3F94A4B700679E97A657BFFF7
:1063F30020222EE50E602A7E008E82758300121BFA
:106403005860060EEE650F70F0C2D5EBC0E0EAC02F
:10641300E0E9C0E0EE12655FD0E0F9D0E0FAD0E049
:10642300FB121B3FFF60AAEBC0E0EAC0E0E9C0E05B
:10643300126306D0E02401F9D0E03400FAD0E0FB87
:10644300E50F0460DCD50FD980877BFF7A65795B24
:10645300D222809C791080027908C226C228800843
:10646300D2D5790A8004790AC2D5E50F047002F502
:106473000FE4FAFDFEFF1262C3FC7B082021131216
:1064830062C3FD7B1030200A1262C3FE1262C3FF97
:106493007B20EC3382D592D55013C3E43020069F82
:1064A300FFE49EFEE42021039DFDE49CFCE4CBF885
:1064B300C221EC700CCFCECDCCE824F8F870F38079
:1064C30017C3EF33FFEE33FEED33FDEC33FCEB3359
:1064D300FB994002FB0FD8E9EB302105F8D0E0C46B
:1064E30048B221C0E00AEC4D4E4F78207B0070C2C9
:1064F300EAB50F0040BCC0E0126561D0F0D0E020E7
:106503002104C4C0E0C4B221C0F01262EFD0F0D5C0
:10651300F0EB0263401220AF63DD5364575863AE60
:106523004C63AA42645B4F64634464634963C3433B
:08653300646955644D46644D96
:10653B0045644D4766095063B22D63B62E63D92B64
:10654B0063BA2363D72065F22A637248000063D1D4
:10655B003F3F3F00790AA2D5202314302509B910FB
:10656B00020404B9080104A2D5202602500104201C
:10657B0022689222B50E005034C0E07F20302319E0
:10658B007F30A22272267225500F1265B8C222C22A
:10659B0026C225C2287F30800F302503E9C0E012C8
:1065AB006306302503D0E0F9D0E0B50ECC302517CB
:1065BB007F30B9100C1263067F583024077F788028
:1065CB0003B908031263063022057F2D0263067F91
:1065DB00202028F87F2B2026F322922280CF286EB2
:1065EB00756C6C2900D2211262C33021F8C221785C
:1065FB000E30D50108F60263722D504349581262D2
:10660B00C32403B405004001E4906604931262F7BF
:0D661B00743A1262F7D223750E0402645720
:10B48E0010320B12B5FABF0D027F0A02B0E890FE21
:04B49E0025E0FF2284
:08B6140090FE25EFF0D2322276
:10B4A200EFC394094005EF940E4004EFB42003D398
:04B4B2008001C32230
:10B0E800EFB40A07740D12B0F3740A309811A899D6
:10B0F800B8130CC2983098FDA899C298B811F630C8
:07B1080099FDC299F599229F
:0AB5FA003098FDAF99C2987E002240
:00000001FF
